
bin\Release\InertialHand.elf:     file format elf32-avr

Sections:
Idx Name          Size      VMA       LMA       File off  Algn
  0 .text         0000148e  00000000  00000000  00000094  2**1
                  CONTENTS, ALLOC, LOAD, READONLY, CODE
  1 .data         000000ec  00802000  0000148e  00001522  2**0
                  CONTENTS, ALLOC, LOAD, DATA
  2 .bss          00000283  008020ec  008020ec  0000160e  2**0
                  ALLOC

Disassembly of section .text:

00000000 <__vectors>:
       0:	0c 94 fa 00 	jmp	0x1f4	; 0x1f4 <__ctors_end>
       4:	0c 94 20 01 	jmp	0x240	; 0x240 <__bad_interrupt>
       8:	0c 94 20 01 	jmp	0x240	; 0x240 <__bad_interrupt>
       c:	0c 94 20 01 	jmp	0x240	; 0x240 <__bad_interrupt>
      10:	0c 94 20 01 	jmp	0x240	; 0x240 <__bad_interrupt>
      14:	0c 94 20 01 	jmp	0x240	; 0x240 <__bad_interrupt>
      18:	0c 94 20 01 	jmp	0x240	; 0x240 <__bad_interrupt>
      1c:	0c 94 20 01 	jmp	0x240	; 0x240 <__bad_interrupt>
      20:	0c 94 20 01 	jmp	0x240	; 0x240 <__bad_interrupt>
      24:	0c 94 20 01 	jmp	0x240	; 0x240 <__bad_interrupt>
      28:	0c 94 20 01 	jmp	0x240	; 0x240 <__bad_interrupt>
      2c:	0c 94 20 01 	jmp	0x240	; 0x240 <__bad_interrupt>
      30:	0c 94 20 01 	jmp	0x240	; 0x240 <__bad_interrupt>
      34:	0c 94 20 01 	jmp	0x240	; 0x240 <__bad_interrupt>
      38:	0c 94 20 01 	jmp	0x240	; 0x240 <__bad_interrupt>
      3c:	0c 94 20 01 	jmp	0x240	; 0x240 <__bad_interrupt>
      40:	0c 94 65 08 	jmp	0x10ca	; 0x10ca <__vector_16>
      44:	0c 94 20 01 	jmp	0x240	; 0x240 <__bad_interrupt>
      48:	0c 94 20 01 	jmp	0x240	; 0x240 <__bad_interrupt>
      4c:	0c 94 20 01 	jmp	0x240	; 0x240 <__bad_interrupt>
      50:	0c 94 20 01 	jmp	0x240	; 0x240 <__bad_interrupt>
      54:	0c 94 20 01 	jmp	0x240	; 0x240 <__bad_interrupt>
      58:	0c 94 20 01 	jmp	0x240	; 0x240 <__bad_interrupt>
      5c:	0c 94 20 01 	jmp	0x240	; 0x240 <__bad_interrupt>
      60:	0c 94 20 01 	jmp	0x240	; 0x240 <__bad_interrupt>
      64:	0c 94 8c 02 	jmp	0x518	; 0x518 <__vector_25>
      68:	0c 94 20 01 	jmp	0x240	; 0x240 <__bad_interrupt>
      6c:	0c 94 20 01 	jmp	0x240	; 0x240 <__bad_interrupt>
      70:	0c 94 20 01 	jmp	0x240	; 0x240 <__bad_interrupt>
      74:	0c 94 20 01 	jmp	0x240	; 0x240 <__bad_interrupt>
      78:	0c 94 20 01 	jmp	0x240	; 0x240 <__bad_interrupt>
      7c:	0c 94 20 01 	jmp	0x240	; 0x240 <__bad_interrupt>
      80:	0c 94 20 01 	jmp	0x240	; 0x240 <__bad_interrupt>
      84:	0c 94 20 01 	jmp	0x240	; 0x240 <__bad_interrupt>
      88:	0c 94 20 01 	jmp	0x240	; 0x240 <__bad_interrupt>
      8c:	0c 94 20 01 	jmp	0x240	; 0x240 <__bad_interrupt>
      90:	0c 94 20 01 	jmp	0x240	; 0x240 <__bad_interrupt>
      94:	0c 94 20 01 	jmp	0x240	; 0x240 <__bad_interrupt>
      98:	0c 94 20 01 	jmp	0x240	; 0x240 <__bad_interrupt>
      9c:	0c 94 20 01 	jmp	0x240	; 0x240 <__bad_interrupt>
      a0:	0c 94 20 01 	jmp	0x240	; 0x240 <__bad_interrupt>
      a4:	0c 94 20 01 	jmp	0x240	; 0x240 <__bad_interrupt>
      a8:	0c 94 20 01 	jmp	0x240	; 0x240 <__bad_interrupt>
      ac:	0c 94 64 03 	jmp	0x6c8	; 0x6c8 <__vector_43>
      b0:	0c 94 20 01 	jmp	0x240	; 0x240 <__bad_interrupt>
      b4:	0c 94 20 01 	jmp	0x240	; 0x240 <__bad_interrupt>
      b8:	0c 94 20 01 	jmp	0x240	; 0x240 <__bad_interrupt>
      bc:	0c 94 20 01 	jmp	0x240	; 0x240 <__bad_interrupt>
      c0:	0c 94 20 01 	jmp	0x240	; 0x240 <__bad_interrupt>
      c4:	0c 94 20 01 	jmp	0x240	; 0x240 <__bad_interrupt>
      c8:	0c 94 20 01 	jmp	0x240	; 0x240 <__bad_interrupt>
      cc:	0c 94 20 01 	jmp	0x240	; 0x240 <__bad_interrupt>
      d0:	0c 94 20 01 	jmp	0x240	; 0x240 <__bad_interrupt>
      d4:	0c 94 20 01 	jmp	0x240	; 0x240 <__bad_interrupt>
      d8:	0c 94 20 01 	jmp	0x240	; 0x240 <__bad_interrupt>
      dc:	0c 94 20 01 	jmp	0x240	; 0x240 <__bad_interrupt>
      e0:	0c 94 20 01 	jmp	0x240	; 0x240 <__bad_interrupt>
      e4:	0c 94 20 01 	jmp	0x240	; 0x240 <__bad_interrupt>
      e8:	0c 94 20 01 	jmp	0x240	; 0x240 <__bad_interrupt>
      ec:	0c 94 20 01 	jmp	0x240	; 0x240 <__bad_interrupt>
      f0:	0c 94 20 01 	jmp	0x240	; 0x240 <__bad_interrupt>
      f4:	0c 94 20 01 	jmp	0x240	; 0x240 <__bad_interrupt>
      f8:	0c 94 20 01 	jmp	0x240	; 0x240 <__bad_interrupt>
      fc:	0c 94 20 01 	jmp	0x240	; 0x240 <__bad_interrupt>
     100:	0c 94 20 01 	jmp	0x240	; 0x240 <__bad_interrupt>
     104:	0c 94 20 01 	jmp	0x240	; 0x240 <__bad_interrupt>
     108:	0c 94 20 01 	jmp	0x240	; 0x240 <__bad_interrupt>
     10c:	0c 94 20 01 	jmp	0x240	; 0x240 <__bad_interrupt>
     110:	0c 94 20 01 	jmp	0x240	; 0x240 <__bad_interrupt>
     114:	0c 94 20 01 	jmp	0x240	; 0x240 <__bad_interrupt>
     118:	0c 94 20 01 	jmp	0x240	; 0x240 <__bad_interrupt>
     11c:	0c 94 20 01 	jmp	0x240	; 0x240 <__bad_interrupt>
     120:	0c 94 20 01 	jmp	0x240	; 0x240 <__bad_interrupt>
     124:	0c 94 20 01 	jmp	0x240	; 0x240 <__bad_interrupt>
     128:	0c 94 20 01 	jmp	0x240	; 0x240 <__bad_interrupt>
     12c:	0c 94 20 01 	jmp	0x240	; 0x240 <__bad_interrupt>
     130:	0c 94 20 01 	jmp	0x240	; 0x240 <__bad_interrupt>
     134:	0c 94 20 01 	jmp	0x240	; 0x240 <__bad_interrupt>
     138:	0c 94 20 01 	jmp	0x240	; 0x240 <__bad_interrupt>
     13c:	0c 94 20 01 	jmp	0x240	; 0x240 <__bad_interrupt>
     140:	0c 94 20 01 	jmp	0x240	; 0x240 <__bad_interrupt>
     144:	0c 94 20 01 	jmp	0x240	; 0x240 <__bad_interrupt>
     148:	0c 94 20 01 	jmp	0x240	; 0x240 <__bad_interrupt>
     14c:	0c 94 20 01 	jmp	0x240	; 0x240 <__bad_interrupt>
     150:	0c 94 20 01 	jmp	0x240	; 0x240 <__bad_interrupt>
     154:	0c 94 20 01 	jmp	0x240	; 0x240 <__bad_interrupt>
     158:	0c 94 20 01 	jmp	0x240	; 0x240 <__bad_interrupt>
     15c:	0c 94 22 01 	jmp	0x244	; 0x244 <__vector_87>
     160:	0c 94 20 01 	jmp	0x240	; 0x240 <__bad_interrupt>
     164:	0c 94 20 01 	jmp	0x240	; 0x240 <__bad_interrupt>
     168:	0c 94 20 01 	jmp	0x240	; 0x240 <__bad_interrupt>
     16c:	0c 94 20 01 	jmp	0x240	; 0x240 <__bad_interrupt>
     170:	0c 94 20 01 	jmp	0x240	; 0x240 <__bad_interrupt>
     174:	0c 94 20 01 	jmp	0x240	; 0x240 <__bad_interrupt>
     178:	0c 94 20 01 	jmp	0x240	; 0x240 <__bad_interrupt>
     17c:	0c 94 20 01 	jmp	0x240	; 0x240 <__bad_interrupt>
     180:	0c 94 20 01 	jmp	0x240	; 0x240 <__bad_interrupt>
     184:	0c 94 20 01 	jmp	0x240	; 0x240 <__bad_interrupt>
     188:	0c 94 20 01 	jmp	0x240	; 0x240 <__bad_interrupt>
     18c:	0c 94 20 01 	jmp	0x240	; 0x240 <__bad_interrupt>
     190:	0c 94 20 01 	jmp	0x240	; 0x240 <__bad_interrupt>
     194:	0c 94 20 01 	jmp	0x240	; 0x240 <__bad_interrupt>
     198:	0c 94 20 01 	jmp	0x240	; 0x240 <__bad_interrupt>
     19c:	0c 94 20 01 	jmp	0x240	; 0x240 <__bad_interrupt>
     1a0:	0c 94 20 01 	jmp	0x240	; 0x240 <__bad_interrupt>
     1a4:	0c 94 20 01 	jmp	0x240	; 0x240 <__bad_interrupt>
     1a8:	0c 94 20 01 	jmp	0x240	; 0x240 <__bad_interrupt>
     1ac:	0c 94 20 01 	jmp	0x240	; 0x240 <__bad_interrupt>
     1b0:	0c 94 20 01 	jmp	0x240	; 0x240 <__bad_interrupt>
     1b4:	0c 94 20 01 	jmp	0x240	; 0x240 <__bad_interrupt>
     1b8:	0c 94 20 01 	jmp	0x240	; 0x240 <__bad_interrupt>
     1bc:	0c 94 20 01 	jmp	0x240	; 0x240 <__bad_interrupt>
     1c0:	0c 94 20 01 	jmp	0x240	; 0x240 <__bad_interrupt>
     1c4:	0c 94 20 01 	jmp	0x240	; 0x240 <__bad_interrupt>
     1c8:	0c 94 20 01 	jmp	0x240	; 0x240 <__bad_interrupt>
     1cc:	0c 94 20 01 	jmp	0x240	; 0x240 <__bad_interrupt>
     1d0:	0c 94 20 01 	jmp	0x240	; 0x240 <__bad_interrupt>
     1d4:	0c 94 20 01 	jmp	0x240	; 0x240 <__bad_interrupt>
     1d8:	0c 94 20 01 	jmp	0x240	; 0x240 <__bad_interrupt>
     1dc:	0c 94 20 01 	jmp	0x240	; 0x240 <__bad_interrupt>
     1e0:	0c 94 20 01 	jmp	0x240	; 0x240 <__bad_interrupt>
     1e4:	0c 94 20 01 	jmp	0x240	; 0x240 <__bad_interrupt>
     1e8:	0c 94 20 01 	jmp	0x240	; 0x240 <__bad_interrupt>
     1ec:	0c 94 20 01 	jmp	0x240	; 0x240 <__bad_interrupt>
     1f0:	0c 94 20 01 	jmp	0x240	; 0x240 <__bad_interrupt>

000001f4 <__ctors_end>:
     1f4:	11 24       	eor	r1, r1
     1f6:	1f be       	out	0x3f, r1	; 63
     1f8:	cf ef       	ldi	r28, 0xFF	; 255
     1fa:	df e3       	ldi	r29, 0x3F	; 63
     1fc:	de bf       	out	0x3e, r29	; 62
     1fe:	cd bf       	out	0x3d, r28	; 61
     200:	00 e0       	ldi	r16, 0x00	; 0
     202:	0c bf       	out	0x3c, r16	; 60
     204:	18 be       	out	0x38, r1	; 56
     206:	19 be       	out	0x39, r1	; 57
     208:	1a be       	out	0x3a, r1	; 58
     20a:	1b be       	out	0x3b, r1	; 59

0000020c <__do_copy_data>:
     20c:	10 e2       	ldi	r17, 0x20	; 32
     20e:	a0 e0       	ldi	r26, 0x00	; 0
     210:	b0 e2       	ldi	r27, 0x20	; 32
     212:	ee e8       	ldi	r30, 0x8E	; 142
     214:	f4 e1       	ldi	r31, 0x14	; 20
     216:	00 e0       	ldi	r16, 0x00	; 0
     218:	0b bf       	out	0x3b, r16	; 59
     21a:	02 c0       	rjmp	.+4      	; 0x220 <__do_copy_data+0x14>
     21c:	07 90       	elpm	r0, Z+
     21e:	0d 92       	st	X+, r0
     220:	ac 3e       	cpi	r26, 0xEC	; 236
     222:	b1 07       	cpc	r27, r17
     224:	d9 f7       	brne	.-10     	; 0x21c <__do_copy_data+0x10>
     226:	1b be       	out	0x3b, r1	; 59

00000228 <__do_clear_bss>:
     228:	13 e2       	ldi	r17, 0x23	; 35
     22a:	ac ee       	ldi	r26, 0xEC	; 236
     22c:	b0 e2       	ldi	r27, 0x20	; 32
     22e:	01 c0       	rjmp	.+2      	; 0x232 <.do_clear_bss_start>

00000230 <.do_clear_bss_loop>:
     230:	1d 92       	st	X+, r1

00000232 <.do_clear_bss_start>:
     232:	af 36       	cpi	r26, 0x6F	; 111
     234:	b1 07       	cpc	r27, r17
     236:	e1 f7       	brne	.-8      	; 0x230 <.do_clear_bss_loop>
     238:	0e 94 f6 07 	call	0xfec	; 0xfec <main>
     23c:	0c 94 45 0a 	jmp	0x148a	; 0x148a <_exit>

00000240 <__bad_interrupt>:
     240:	0c 94 50 03 	jmp	0x6a0	; 0x6a0 <__vector_default>

00000244 <__vector_87>:
     244:	1f 92       	push	r1
     246:	0f 92       	push	r0
     248:	0f b6       	in	r0, 0x3f	; 63
     24a:	0f 92       	push	r0
     24c:	08 b6       	in	r0, 0x38	; 56
     24e:	0f 92       	push	r0
     250:	0b b6       	in	r0, 0x3b	; 59
     252:	0f 92       	push	r0
     254:	11 24       	eor	r1, r1
     256:	18 be       	out	0x38, r1	; 56
     258:	1b be       	out	0x3b, r1	; 59
     25a:	8f 93       	push	r24
     25c:	9f 93       	push	r25
     25e:	ef 93       	push	r30
     260:	ff 93       	push	r31
     262:	88 e0       	ldi	r24, 0x08	; 8
     264:	e0 e6       	ldi	r30, 0x60	; 96
     266:	f6 e0       	ldi	r31, 0x06	; 6
     268:	86 83       	std	Z+6, r24	; 0x06
     26a:	80 91 c3 09 	lds	r24, 0x09C3
     26e:	e0 91 21 20 	lds	r30, 0x2021
     272:	f0 e0       	ldi	r31, 0x00	; 0
     274:	e0 50       	subi	r30, 0x00	; 0
     276:	f0 4e       	sbci	r31, 0xE0	; 224
     278:	80 83       	st	Z, r24
     27a:	80 91 21 20 	lds	r24, 0x2021
     27e:	8e 31       	cpi	r24, 0x1E	; 30
     280:	28 f4       	brcc	.+10     	; 0x28c <__vector_87+0x48>
     282:	80 91 21 20 	lds	r24, 0x2021
     286:	8f 5f       	subi	r24, 0xFF	; 255
     288:	80 93 21 20 	sts	0x2021, r24
     28c:	80 91 20 20 	lds	r24, 0x2020
     290:	81 50       	subi	r24, 0x01	; 1
     292:	80 93 20 20 	sts	0x2020, r24
     296:	80 91 20 20 	lds	r24, 0x2020
     29a:	88 23       	and	r24, r24
     29c:	31 f5       	brne	.+76     	; 0x2ea <__vector_87+0xa6>
     29e:	81 e0       	ldi	r24, 0x01	; 1
     2a0:	80 93 1e 20 	sts	0x201E, r24
     2a4:	80 91 22 20 	lds	r24, 0x2022
     2a8:	90 91 23 20 	lds	r25, 0x2023
     2ac:	89 2b       	or	r24, r25
     2ae:	91 f4       	brne	.+36     	; 0x2d4 <__vector_87+0x90>
     2b0:	80 91 c0 09 	lds	r24, 0x09C0
     2b4:	8f 7b       	andi	r24, 0xBF	; 191
     2b6:	80 93 c0 09 	sts	0x09C0, r24
     2ba:	80 e8       	ldi	r24, 0x80	; 128
     2bc:	e0 e6       	ldi	r30, 0x60	; 96
     2be:	f6 e0       	ldi	r31, 0x06	; 6
     2c0:	85 83       	std	Z+5, r24	; 0x05
     2c2:	82 e0       	ldi	r24, 0x02	; 2
     2c4:	80 93 00 09 	sts	0x0900, r24
     2c8:	80 91 01 09 	lds	r24, 0x0901
     2cc:	80 61       	ori	r24, 0x10	; 16
     2ce:	e0 e0       	ldi	r30, 0x00	; 0
     2d0:	f9 e0       	ldi	r31, 0x09	; 9
     2d2:	81 83       	std	Z+1, r24	; 0x01
     2d4:	80 91 22 20 	lds	r24, 0x2022
     2d8:	90 91 23 20 	lds	r25, 0x2023
     2dc:	01 97       	sbiw	r24, 0x01	; 1
     2de:	71 f4       	brne	.+28     	; 0x2fc <__vector_87+0xb8>
     2e0:	80 e1       	ldi	r24, 0x10	; 16
     2e2:	e0 e6       	ldi	r30, 0x60	; 96
     2e4:	f6 e0       	ldi	r31, 0x06	; 6
     2e6:	85 83       	std	Z+5, r24	; 0x05
     2e8:	09 c0       	rjmp	.+18     	; 0x2fc <__vector_87+0xb8>
     2ea:	e0 91 21 20 	lds	r30, 0x2021
     2ee:	f0 e0       	ldi	r31, 0x00	; 0
     2f0:	e0 50       	subi	r30, 0x00	; 0
     2f2:	f0 4e       	sbci	r31, 0xE0	; 224
     2f4:	80 81       	ld	r24, Z
     2f6:	e0 ec       	ldi	r30, 0xC0	; 192
     2f8:	f9 e0       	ldi	r31, 0x09	; 9
     2fa:	83 83       	std	Z+3, r24	; 0x03
     2fc:	ff 91       	pop	r31
     2fe:	ef 91       	pop	r30
     300:	9f 91       	pop	r25
     302:	8f 91       	pop	r24
     304:	0f 90       	pop	r0
     306:	0b be       	out	0x3b, r0	; 59
     308:	0f 90       	pop	r0
     30a:	08 be       	out	0x38, r0	; 56
     30c:	0f 90       	pop	r0
     30e:	0f be       	out	0x3f, r0	; 63
     310:	0f 90       	pop	r0
     312:	1f 90       	pop	r1
     314:	18 95       	reti

00000316 <SPIbufferpointer>:
     316:	80 e0       	ldi	r24, 0x00	; 0
     318:	90 e2       	ldi	r25, 0x20	; 32
     31a:	08 95       	ret

0000031c <SPITransferReady>:
     31c:	80 91 1e 20 	lds	r24, 0x201E
     320:	08 95       	ret

00000322 <SPIBufferAvailable>:
     322:	80 91 1f 20 	lds	r24, 0x201F
     326:	08 95       	ret

00000328 <SPITarget>:
     328:	20 91 22 20 	lds	r18, 0x2022
     32c:	30 91 23 20 	lds	r19, 0x2023
     330:	c9 01       	movw	r24, r18
     332:	08 95       	ret

00000334 <SPIClearBuffer>:
     334:	80 91 1e 20 	lds	r24, 0x201E
     338:	88 23       	and	r24, r24
     33a:	19 f0       	breq	.+6      	; 0x342 <SPIClearBuffer+0xe>
     33c:	81 e0       	ldi	r24, 0x01	; 1
     33e:	80 93 1f 20 	sts	0x201F, r24
     342:	08 95       	ret

00000344 <SPI_DAC_2636_init>:
     344:	e0 ec       	ldi	r30, 0xC0	; 192
     346:	f9 e0       	ldi	r31, 0x09	; 9
     348:	8d ed       	ldi	r24, 0xDD	; 221
     34a:	80 83       	st	Z, r24
     34c:	83 e0       	ldi	r24, 0x03	; 3
     34e:	81 83       	std	Z+1, r24	; 0x01
     350:	08 95       	ret

00000352 <InitADCClock>:
     352:	e0 e0       	ldi	r30, 0x00	; 0
     354:	f9 e0       	ldi	r31, 0x09	; 9
     356:	82 e0       	ldi	r24, 0x02	; 2
     358:	80 83       	st	Z, r24
     35a:	81 e1       	ldi	r24, 0x11	; 17
     35c:	81 83       	std	Z+1, r24	; 0x01
     35e:	12 82       	std	Z+2, r1	; 0x02
     360:	13 82       	std	Z+3, r1	; 0x03
     362:	14 82       	std	Z+4, r1	; 0x04
     364:	16 82       	std	Z+6, r1	; 0x06
     366:	17 82       	std	Z+7, r1	; 0x07
     368:	82 e0       	ldi	r24, 0x02	; 2
     36a:	90 e0       	ldi	r25, 0x00	; 0
     36c:	80 a7       	std	Z+40, r24	; 0x28
     36e:	91 a7       	std	Z+41, r25	; 0x29
     370:	08 95       	ret

00000372 <SPI_ADC_1408_init>:
     372:	80 91 ec 20 	lds	r24, 0x20EC
     376:	88 23       	and	r24, r24
     378:	29 f4       	brne	.+10     	; 0x384 <SPI_ADC_1408_init+0x12>
     37a:	0e 94 a9 01 	call	0x352	; 0x352 <InitADCClock>
     37e:	81 e0       	ldi	r24, 0x01	; 1
     380:	80 93 ec 20 	sts	0x20EC, r24
     384:	89 e5       	ldi	r24, 0x59	; 89
     386:	80 93 c0 09 	sts	0x09C0, r24
     38a:	83 e0       	ldi	r24, 0x03	; 3
     38c:	e0 ec       	ldi	r30, 0xC0	; 192
     38e:	f9 e0       	ldi	r31, 0x09	; 9
     390:	81 83       	std	Z+1, r24	; 0x01
     392:	08 95       	ret

00000394 <SPITransceiveArray>:
     394:	df 92       	push	r13
     396:	ef 92       	push	r14
     398:	ff 92       	push	r15
     39a:	0f 93       	push	r16
     39c:	1f 93       	push	r17
     39e:	df 93       	push	r29
     3a0:	cf 93       	push	r28
     3a2:	0f 92       	push	r0
     3a4:	cd b7       	in	r28, 0x3d	; 61
     3a6:	de b7       	in	r29, 0x3e	; 62
     3a8:	e8 2e       	mov	r14, r24
     3aa:	d9 2e       	mov	r13, r25
     3ac:	f6 2e       	mov	r15, r22
     3ae:	80 91 1f 20 	lds	r24, 0x201F
     3b2:	88 23       	and	r24, r24
     3b4:	11 f4       	brne	.+4      	; 0x3ba <SPITransceiveArray+0x26>
     3b6:	82 e0       	ldi	r24, 0x02	; 2
     3b8:	57 c0       	rjmp	.+174    	; 0x468 <SPITransceiveArray+0xd4>
     3ba:	8d e1       	ldi	r24, 0x1D	; 29
     3bc:	86 17       	cp	r24, r22
     3be:	10 f4       	brcc	.+4      	; 0x3c4 <SPITransceiveArray+0x30>
     3c0:	81 e0       	ldi	r24, 0x01	; 1
     3c2:	52 c0       	rjmp	.+164    	; 0x468 <SPITransceiveArray+0xd4>
     3c4:	10 92 1f 20 	sts	0x201F, r1
     3c8:	10 92 1e 20 	sts	0x201E, r1
     3cc:	84 2f       	mov	r24, r20
     3ce:	90 e0       	ldi	r25, 0x00	; 0
     3d0:	80 93 22 20 	sts	0x2022, r24
     3d4:	90 93 23 20 	sts	0x2023, r25
     3d8:	60 93 20 20 	sts	0x2020, r22
     3dc:	10 92 21 20 	sts	0x2021, r1
     3e0:	80 91 c0 09 	lds	r24, 0x09C0
     3e4:	80 64       	ori	r24, 0x40	; 64
     3e6:	80 93 c0 09 	sts	0x09C0, r24
     3ea:	44 23       	and	r20, r20
     3ec:	19 f0       	breq	.+6      	; 0x3f4 <SPITransceiveArray+0x60>
     3ee:	41 30       	cpi	r20, 0x01	; 1
     3f0:	29 f5       	brne	.+74     	; 0x43c <SPITransceiveArray+0xa8>
     3f2:	1d c0       	rjmp	.+58     	; 0x42e <SPITransceiveArray+0x9a>
     3f4:	10 92 00 09 	sts	0x0900, r1
     3f8:	80 91 01 09 	lds	r24, 0x0901
     3fc:	8f 7e       	andi	r24, 0xEF	; 239
     3fe:	e0 e0       	ldi	r30, 0x00	; 0
     400:	f9 e0       	ldi	r31, 0x09	; 9
     402:	81 83       	std	Z+1, r24	; 0x01
     404:	00 e6       	ldi	r16, 0x60	; 96
     406:	16 e0       	ldi	r17, 0x06	; 6
     408:	91 e0       	ldi	r25, 0x01	; 1
     40a:	f8 01       	movw	r30, r16
     40c:	96 83       	std	Z+6, r25	; 0x06
     40e:	99 83       	std	Y+1, r25	; 0x01
     410:	0e 94 b9 01 	call	0x372	; 0x372 <SPI_ADC_1408_init>
     414:	88 e0       	ldi	r24, 0x08	; 8
     416:	f8 01       	movw	r30, r16
     418:	85 83       	std	Z+5, r24	; 0x05
     41a:	99 81       	ldd	r25, Y+1	; 0x01
     41c:	89 2f       	mov	r24, r25
     41e:	8a 95       	dec	r24
     420:	f1 f7       	brne	.-4      	; 0x41e <SPITransceiveArray+0x8a>
     422:	96 83       	std	Z+6, r25	; 0x06
     424:	89 2f       	mov	r24, r25
     426:	8a 95       	dec	r24
     428:	f1 f7       	brne	.-4      	; 0x426 <SPITransceiveArray+0x92>
     42a:	95 83       	std	Z+5, r25	; 0x05
     42c:	07 c0       	rjmp	.+14     	; 0x43c <SPITransceiveArray+0xa8>
     42e:	8d ed       	ldi	r24, 0xDD	; 221
     430:	80 93 c0 09 	sts	0x09C0, r24
     434:	83 e0       	ldi	r24, 0x03	; 3
     436:	e0 ec       	ldi	r30, 0xC0	; 192
     438:	f9 e0       	ldi	r31, 0x09	; 9
     43a:	81 83       	std	Z+1, r24	; 0x01
     43c:	8e 2d       	mov	r24, r14
     43e:	9d 2d       	mov	r25, r13
     440:	9c 01       	movw	r18, r24
     442:	d9 01       	movw	r26, r18
     444:	20 e0       	ldi	r18, 0x00	; 0
     446:	30 e0       	ldi	r19, 0x00	; 0
     448:	07 c0       	rjmp	.+14     	; 0x458 <SPITransceiveArray+0xc4>
     44a:	8d 91       	ld	r24, X+
     44c:	f9 01       	movw	r30, r18
     44e:	e0 50       	subi	r30, 0x00	; 0
     450:	f0 4e       	sbci	r31, 0xE0	; 224
     452:	80 83       	st	Z, r24
     454:	2f 5f       	subi	r18, 0xFF	; 255
     456:	3f 4f       	sbci	r19, 0xFF	; 255
     458:	2f 15       	cp	r18, r15
     45a:	b8 f3       	brcs	.-18     	; 0x44a <SPITransceiveArray+0xb6>
     45c:	80 91 00 20 	lds	r24, 0x2000
     460:	e0 ec       	ldi	r30, 0xC0	; 192
     462:	f9 e0       	ldi	r31, 0x09	; 9
     464:	83 83       	std	Z+3, r24	; 0x03
     466:	80 e0       	ldi	r24, 0x00	; 0
     468:	0f 90       	pop	r0
     46a:	cf 91       	pop	r28
     46c:	df 91       	pop	r29
     46e:	1f 91       	pop	r17
     470:	0f 91       	pop	r16
     472:	ff 90       	pop	r15
     474:	ef 90       	pop	r14
     476:	df 90       	pop	r13
     478:	08 95       	ret

0000047a <SPI_SendByte>:
     47a:	fc 01       	movw	r30, r24
     47c:	63 83       	std	Z+3, r22	; 0x03
     47e:	08 95       	ret

00000480 <SPI_RecvByte>:
     480:	fc 01       	movw	r30, r24
     482:	83 81       	ldd	r24, Z+3	; 0x03
     484:	08 95       	ret

00000486 <DAC_2636SelectRef>:
     486:	81 e0       	ldi	r24, 0x01	; 1
     488:	08 95       	ret

0000048a <DAC_2636WriteSingleChannel>:
     48a:	df 93       	push	r29
     48c:	cf 93       	push	r28
     48e:	00 d0       	rcall	.+0      	; 0x490 <DAC_2636WriteSingleChannel+0x6>
     490:	cd b7       	in	r28, 0x3d	; 61
     492:	de b7       	in	r29, 0x3e	; 62
     494:	9c 01       	movw	r18, r24
     496:	67 30       	cpi	r22, 0x07	; 7
     498:	10 f0       	brcs	.+4      	; 0x49e <DAC_2636WriteSingleChannel+0x14>
     49a:	91 e0       	ldi	r25, 0x01	; 1
     49c:	19 c0       	rjmp	.+50     	; 0x4d0 <DAC_2636WriteSingleChannel+0x46>
     49e:	60 63       	ori	r22, 0x30	; 48
     4a0:	69 83       	std	Y+1, r22	; 0x01
     4a2:	34 e0       	ldi	r19, 0x04	; 4
     4a4:	96 95       	lsr	r25
     4a6:	87 95       	ror	r24
     4a8:	3a 95       	dec	r19
     4aa:	e1 f7       	brne	.-8      	; 0x4a4 <DAC_2636WriteSingleChannel+0x1a>
     4ac:	8a 83       	std	Y+2, r24	; 0x02
     4ae:	82 2f       	mov	r24, r18
     4b0:	82 95       	swap	r24
     4b2:	80 7f       	andi	r24, 0xF0	; 240
     4b4:	8b 83       	std	Y+3, r24	; 0x03
     4b6:	ce 01       	movw	r24, r28
     4b8:	01 96       	adiw	r24, 0x01	; 1
     4ba:	63 e0       	ldi	r22, 0x03	; 3
     4bc:	41 e0       	ldi	r20, 0x01	; 1
     4be:	0e 94 ca 01 	call	0x394	; 0x394 <SPITransceiveArray>
     4c2:	98 2f       	mov	r25, r24
     4c4:	88 23       	and	r24, r24
     4c6:	21 f4       	brne	.+8      	; 0x4d0 <DAC_2636WriteSingleChannel+0x46>
     4c8:	80 e1       	ldi	r24, 0x10	; 16
     4ca:	e0 e6       	ldi	r30, 0x60	; 96
     4cc:	f6 e0       	ldi	r31, 0x06	; 6
     4ce:	86 83       	std	Z+6, r24	; 0x06
     4d0:	89 2f       	mov	r24, r25
     4d2:	23 96       	adiw	r28, 0x03	; 3
     4d4:	cd bf       	out	0x3d, r28	; 61
     4d6:	de bf       	out	0x3e, r29	; 62
     4d8:	cf 91       	pop	r28
     4da:	df 91       	pop	r29
     4dc:	08 95       	ret

000004de <DAC_2636_init>:
     4de:	e0 e6       	ldi	r30, 0x60	; 96
     4e0:	f6 e0       	ldi	r31, 0x06	; 6
     4e2:	80 eb       	ldi	r24, 0xB0	; 176
     4e4:	81 83       	std	Z+1, r24	; 0x01
     4e6:	80 e1       	ldi	r24, 0x10	; 16
     4e8:	85 83       	std	Z+5, r24	; 0x05
     4ea:	86 e0       	ldi	r24, 0x06	; 6
     4ec:	81 83       	std	Z+1, r24	; 0x01
     4ee:	82 e0       	ldi	r24, 0x02	; 2
     4f0:	85 83       	std	Z+5, r24	; 0x05
     4f2:	84 e0       	ldi	r24, 0x04	; 4
     4f4:	85 83       	std	Z+5, r24	; 0x05
     4f6:	08 95       	ret

000004f8 <ADC_1408_init>:
     4f8:	e0 e6       	ldi	r30, 0x60	; 96
     4fa:	f6 e0       	ldi	r31, 0x06	; 6
     4fc:	89 e0       	ldi	r24, 0x09	; 9
     4fe:	81 83       	std	Z+1, r24	; 0x01
     500:	98 e0       	ldi	r25, 0x08	; 8
     502:	96 83       	std	Z+6, r25	; 0x06
     504:	81 e0       	ldi	r24, 0x01	; 1
     506:	85 83       	std	Z+5, r24	; 0x05
     508:	e0 e8       	ldi	r30, 0x80	; 128
     50a:	f6 e0       	ldi	r31, 0x06	; 6
     50c:	8f e0       	ldi	r24, 0x0F	; 15
     50e:	81 83       	std	Z+1, r24	; 0x01
     510:	85 e0       	ldi	r24, 0x05	; 5
     512:	85 83       	std	Z+5, r24	; 0x05
     514:	95 83       	std	Z+5, r25	; 0x05
     516:	08 95       	ret

00000518 <__vector_25>:
     518:	1f 92       	push	r1
     51a:	0f 92       	push	r0
     51c:	0f b6       	in	r0, 0x3f	; 63
     51e:	0f 92       	push	r0
     520:	08 b6       	in	r0, 0x38	; 56
     522:	0f 92       	push	r0
     524:	0b b6       	in	r0, 0x3b	; 59
     526:	0f 92       	push	r0
     528:	11 24       	eor	r1, r1
     52a:	18 be       	out	0x38, r1	; 56
     52c:	1b be       	out	0x3b, r1	; 59
     52e:	8f 93       	push	r24
     530:	ef 93       	push	r30
     532:	ff 93       	push	r31
     534:	e0 91 5e 21 	lds	r30, 0x215E
     538:	80 91 a0 08 	lds	r24, 0x08A0
     53c:	f0 e0       	ldi	r31, 0x00	; 0
     53e:	e0 5a       	subi	r30, 0xA0	; 160
     540:	fe 4d       	sbci	r31, 0xDE	; 222
     542:	80 83       	st	Z, r24
     544:	80 91 5e 21 	lds	r24, 0x215E
     548:	88 32       	cpi	r24, 0x28	; 40
     54a:	50 f4       	brcc	.+20     	; 0x560 <__vector_25+0x48>
     54c:	80 91 33 21 	lds	r24, 0x2133
     550:	88 32       	cpi	r24, 0x28	; 40
     552:	30 f4       	brcc	.+12     	; 0x560 <__vector_25+0x48>
     554:	80 91 5e 21 	lds	r24, 0x215E
     558:	8f 5f       	subi	r24, 0xFF	; 255
     55a:	80 93 5e 21 	sts	0x215E, r24
     55e:	02 c0       	rjmp	.+4      	; 0x564 <__vector_25+0x4c>
     560:	10 92 5e 21 	sts	0x215E, r1
     564:	80 91 33 21 	lds	r24, 0x2133
     568:	8f 5f       	subi	r24, 0xFF	; 255
     56a:	80 93 33 21 	sts	0x2133, r24
     56e:	ff 91       	pop	r31
     570:	ef 91       	pop	r30
     572:	8f 91       	pop	r24
     574:	0f 90       	pop	r0
     576:	0b be       	out	0x3b, r0	; 59
     578:	0f 90       	pop	r0
     57a:	08 be       	out	0x38, r0	; 56
     57c:	0f 90       	pop	r0
     57e:	0f be       	out	0x3f, r0	; 63
     580:	0f 90       	pop	r0
     582:	1f 90       	pop	r1
     584:	18 95       	reti

00000586 <USBUartRXQuelength>:
     586:	80 91 33 21 	lds	r24, 0x2133
     58a:	08 95       	ret

0000058c <USBUartReadByteFromBuffer>:
     58c:	80 91 5d 21 	lds	r24, 0x215D
     590:	e8 2f       	mov	r30, r24
     592:	f0 e0       	ldi	r31, 0x00	; 0
     594:	e0 5a       	subi	r30, 0xA0	; 160
     596:	fe 4d       	sbci	r31, 0xDE	; 222
     598:	e0 81       	ld	r30, Z
     59a:	88 32       	cpi	r24, 0x28	; 40
     59c:	20 f4       	brcc	.+8      	; 0x5a6 <USBUartReadByteFromBuffer+0x1a>
     59e:	8f 5f       	subi	r24, 0xFF	; 255
     5a0:	80 93 5d 21 	sts	0x215D, r24
     5a4:	02 c0       	rjmp	.+4      	; 0x5aa <USBUartReadByteFromBuffer+0x1e>
     5a6:	10 92 5d 21 	sts	0x215D, r1
     5aa:	80 91 33 21 	lds	r24, 0x2133
     5ae:	88 23       	and	r24, r24
     5b0:	29 f0       	breq	.+10     	; 0x5bc <USBUartReadByteFromBuffer+0x30>
     5b2:	80 91 33 21 	lds	r24, 0x2133
     5b6:	81 50       	subi	r24, 0x01	; 1
     5b8:	80 93 33 21 	sts	0x2133, r24
     5bc:	8e 2f       	mov	r24, r30
     5be:	08 95       	ret

000005c0 <USBUartSendArray>:
     5c0:	9c 01       	movw	r18, r24
     5c2:	80 91 a1 08 	lds	r24, 0x08A1
     5c6:	85 ff       	sbrs	r24, 5
     5c8:	fc cf       	rjmp	.-8      	; 0x5c2 <USBUartSendArray+0x2>
     5ca:	86 2f       	mov	r24, r22
     5cc:	90 e0       	ldi	r25, 0x00	; 0
     5ce:	e0 e0       	ldi	r30, 0x00	; 0
     5d0:	f1 e0       	ldi	r31, 0x01	; 1
     5d2:	84 a3       	std	Z+36, r24	; 0x24
     5d4:	95 a3       	std	Z+37, r25	; 0x25
     5d6:	c9 01       	movw	r24, r18
     5d8:	20 a7       	std	Z+40, r18	; 0x28
     5da:	aa 27       	eor	r26, r26
     5dc:	97 fd       	sbrc	r25, 7
     5de:	a0 95       	com	r26
     5e0:	ba 2f       	mov	r27, r26
     5e2:	29 2f       	mov	r18, r25
     5e4:	3a 2f       	mov	r19, r26
     5e6:	4b 2f       	mov	r20, r27
     5e8:	55 27       	eor	r21, r21
     5ea:	21 a7       	std	Z+41, r18	; 0x29
     5ec:	cd 01       	movw	r24, r26
     5ee:	aa 27       	eor	r26, r26
     5f0:	bb 27       	eor	r27, r27
     5f2:	82 a7       	std	Z+42, r24	; 0x2a
     5f4:	80 91 20 01 	lds	r24, 0x0120
     5f8:	80 68       	ori	r24, 0x80	; 128
     5fa:	80 a3       	std	Z+32, r24	; 0x20
     5fc:	08 95       	ret

000005fe <USBUartSendArray_P>:
     5fe:	9c 01       	movw	r18, r24
     600:	80 91 a1 08 	lds	r24, 0x08A1
     604:	85 ff       	sbrs	r24, 5
     606:	fc cf       	rjmp	.-8      	; 0x600 <USBUartSendArray_P+0x2>
     608:	e0 e0       	ldi	r30, 0x00	; 0
     60a:	f1 e0       	ldi	r31, 0x01	; 1
     60c:	80 91 04 01 	lds	r24, 0x0104
     610:	85 fd       	sbrc	r24, 5
     612:	f6 cf       	rjmp	.-20     	; 0x600 <USBUartSendArray_P+0x2>
     614:	86 2f       	mov	r24, r22
     616:	90 e0       	ldi	r25, 0x00	; 0
     618:	84 a3       	std	Z+36, r24	; 0x24
     61a:	95 a3       	std	Z+37, r25	; 0x25
     61c:	c9 01       	movw	r24, r18
     61e:	20 a7       	std	Z+40, r18	; 0x28
     620:	aa 27       	eor	r26, r26
     622:	97 fd       	sbrc	r25, 7
     624:	a0 95       	com	r26
     626:	ba 2f       	mov	r27, r26
     628:	29 2f       	mov	r18, r25
     62a:	3a 2f       	mov	r19, r26
     62c:	4b 2f       	mov	r20, r27
     62e:	55 27       	eor	r21, r21
     630:	21 a7       	std	Z+41, r18	; 0x29
     632:	cd 01       	movw	r24, r26
     634:	aa 27       	eor	r26, r26
     636:	bb 27       	eor	r27, r27
     638:	82 a7       	std	Z+42, r24	; 0x2a
     63a:	80 91 20 01 	lds	r24, 0x0120
     63e:	80 68       	ori	r24, 0x80	; 128
     640:	80 a3       	std	Z+32, r24	; 0x20
     642:	08 95       	ret

00000644 <USBUartDMASetup>:
     644:	e0 e0       	ldi	r30, 0x00	; 0
     646:	f1 e0       	ldi	r31, 0x01	; 1
     648:	84 e0       	ldi	r24, 0x04	; 4
     64a:	80 a3       	std	Z+32, r24	; 0x20
     64c:	11 a2       	std	Z+33, r1	; 0x21
     64e:	80 e1       	ldi	r24, 0x10	; 16
     650:	82 a3       	std	Z+34, r24	; 0x22
     652:	8c e4       	ldi	r24, 0x4C	; 76
     654:	83 a3       	std	Z+35, r24	; 0x23
     656:	16 a2       	std	Z+38, r1	; 0x26
     658:	80 ea       	ldi	r24, 0xA0	; 160
     65a:	84 a7       	std	Z+44, r24	; 0x2c
     65c:	88 e0       	ldi	r24, 0x08	; 8
     65e:	85 a7       	std	Z+45, r24	; 0x2d
     660:	16 a6       	std	Z+46, r1	; 0x2e
     662:	08 95       	ret

00000664 <USBUartInit>:
     664:	10 92 5d 21 	sts	0x215D, r1
     668:	10 92 5e 21 	sts	0x215E, r1
     66c:	10 92 33 21 	sts	0x2133, r1
     670:	e0 ea       	ldi	r30, 0xA0	; 160
     672:	f8 e0       	ldi	r31, 0x08	; 8
     674:	80 e3       	ldi	r24, 0x30	; 48
     676:	83 83       	std	Z+3, r24	; 0x03
     678:	88 e1       	ldi	r24, 0x18	; 24
     67a:	84 83       	std	Z+4, r24	; 0x04
     67c:	83 e0       	ldi	r24, 0x03	; 3
     67e:	85 83       	std	Z+5, r24	; 0x05
     680:	81 e2       	ldi	r24, 0x21	; 33
     682:	86 83       	std	Z+6, r24	; 0x06
     684:	80 ef       	ldi	r24, 0xF0	; 240
     686:	87 83       	std	Z+7, r24	; 0x07
     688:	08 95       	ret

0000068a <USBUartSendByte>:
     68a:	98 2f       	mov	r25, r24
     68c:	80 91 a1 08 	lds	r24, 0x08A1
     690:	85 fd       	sbrc	r24, 5
     692:	02 c0       	rjmp	.+4      	; 0x698 <USBUartSendByte+0xe>
     694:	81 e0       	ldi	r24, 0x01	; 1
     696:	08 95       	ret
     698:	90 93 a0 08 	sts	0x08A0, r25
     69c:	80 e0       	ldi	r24, 0x00	; 0
     69e:	08 95       	ret

000006a0 <__vector_default>:
     6a0:	1f 92       	push	r1
     6a2:	0f 92       	push	r0
     6a4:	0f b6       	in	r0, 0x3f	; 63
     6a6:	0f 92       	push	r0
     6a8:	08 b6       	in	r0, 0x38	; 56
     6aa:	0f 92       	push	r0
     6ac:	11 24       	eor	r1, r1
     6ae:	18 be       	out	0x38, r1	; 56
     6b0:	8f 93       	push	r24
     6b2:	81 e0       	ldi	r24, 0x01	; 1
     6b4:	80 93 6a 23 	sts	0x236A, r24
     6b8:	8f 91       	pop	r24
     6ba:	0f 90       	pop	r0
     6bc:	08 be       	out	0x38, r0	; 56
     6be:	0f 90       	pop	r0
     6c0:	0f be       	out	0x3f, r0	; 63
     6c2:	0f 90       	pop	r0
     6c4:	1f 90       	pop	r1
     6c6:	18 95       	reti

000006c8 <__vector_43>:
     6c8:	1f 92       	push	r1
     6ca:	0f 92       	push	r0
     6cc:	0f b6       	in	r0, 0x3f	; 63
     6ce:	0f 92       	push	r0
     6d0:	08 b6       	in	r0, 0x38	; 56
     6d2:	0f 92       	push	r0
     6d4:	11 24       	eor	r1, r1
     6d6:	18 be       	out	0x38, r1	; 56
     6d8:	00 00       	nop
     6da:	0f 90       	pop	r0
     6dc:	08 be       	out	0x38, r0	; 56
     6de:	0f 90       	pop	r0
     6e0:	0f be       	out	0x3f, r0	; 63
     6e2:	0f 90       	pop	r0
     6e4:	1f 90       	pop	r1
     6e6:	18 95       	reti

000006e8 <EnableDMA>:
     6e8:	83 e8       	ldi	r24, 0x83	; 131
     6ea:	80 93 00 01 	sts	0x0100, r24
     6ee:	08 95       	ret

000006f0 <ConvertADCResults>:
     6f0:	df 93       	push	r29
     6f2:	cf 93       	push	r28
     6f4:	0f 92       	push	r0
     6f6:	0f 92       	push	r0
     6f8:	cd b7       	in	r28, 0x3d	; 61
     6fa:	de b7       	in	r29, 0x3e	; 62
     6fc:	dc 01       	movw	r26, r24
     6fe:	40 e0       	ldi	r20, 0x00	; 0
     700:	50 e0       	ldi	r21, 0x00	; 0
     702:	3c 91       	ld	r19, X
     704:	20 e0       	ldi	r18, 0x00	; 0
     706:	11 96       	adiw	r26, 0x01	; 1
     708:	8c 91       	ld	r24, X
     70a:	11 97       	sbiw	r26, 0x01	; 1
     70c:	f9 01       	movw	r30, r18
     70e:	e8 0f       	add	r30, r24
     710:	f1 1d       	adc	r31, r1
     712:	e9 83       	std	Y+1, r30	; 0x01
     714:	fa 83       	std	Y+2, r31	; 0x02
     716:	89 81       	ldd	r24, Y+1	; 0x01
     718:	9a 81       	ldd	r25, Y+2	; 0x02
     71a:	88 0f       	add	r24, r24
     71c:	99 1f       	adc	r25, r25
     71e:	88 0f       	add	r24, r24
     720:	99 1f       	adc	r25, r25
     722:	89 83       	std	Y+1, r24	; 0x01
     724:	9a 83       	std	Y+2, r25	; 0x02
     726:	89 81       	ldd	r24, Y+1	; 0x01
     728:	9a 81       	ldd	r25, Y+2	; 0x02
     72a:	95 95       	asr	r25
     72c:	87 95       	ror	r24
     72e:	95 95       	asr	r25
     730:	87 95       	ror	r24
     732:	89 83       	std	Y+1, r24	; 0x01
     734:	9a 83       	std	Y+2, r25	; 0x02
     736:	89 81       	ldd	r24, Y+1	; 0x01
     738:	9a 81       	ldd	r25, Y+2	; 0x02
     73a:	fb 01       	movw	r30, r22
     73c:	e4 0f       	add	r30, r20
     73e:	f5 1f       	adc	r31, r21
     740:	80 83       	st	Z, r24
     742:	91 83       	std	Z+1, r25	; 0x01
     744:	12 96       	adiw	r26, 0x02	; 2
     746:	4e 5f       	subi	r20, 0xFE	; 254
     748:	5f 4f       	sbci	r21, 0xFF	; 255
     74a:	4c 30       	cpi	r20, 0x0C	; 12
     74c:	51 05       	cpc	r21, r1
     74e:	c9 f6       	brne	.-78     	; 0x702 <ConvertADCResults+0x12>
     750:	0f 90       	pop	r0
     752:	0f 90       	pop	r0
     754:	cf 91       	pop	r28
     756:	df 91       	pop	r29
     758:	08 95       	ret

0000075a <InitPorts>:
     75a:	e0 e0       	ldi	r30, 0x00	; 0
     75c:	f6 e0       	ldi	r31, 0x06	; 6
     75e:	10 82       	st	Z, r1
     760:	31 e0       	ldi	r19, 0x01	; 1
     762:	31 83       	std	Z+1, r19	; 0x01
     764:	92 e0       	ldi	r25, 0x02	; 2
     766:	91 83       	std	Z+1, r25	; 0x01
     768:	83 e0       	ldi	r24, 0x03	; 3
     76a:	84 83       	std	Z+4, r24	; 0x04
     76c:	e0 e2       	ldi	r30, 0x20	; 32
     76e:	f6 e0       	ldi	r31, 0x06	; 6
     770:	10 82       	st	Z, r1
     772:	14 82       	std	Z+4, r1	; 0x04
     774:	e0 e4       	ldi	r30, 0x40	; 64
     776:	f6 e0       	ldi	r31, 0x06	; 6
     778:	10 82       	st	Z, r1
     77a:	94 83       	std	Z+4, r25	; 0x04
     77c:	91 83       	std	Z+1, r25	; 0x01
     77e:	28 e0       	ldi	r18, 0x08	; 8
     780:	21 83       	std	Z+1, r18	; 0x01
     782:	e0 e6       	ldi	r30, 0x60	; 96
     784:	f6 e0       	ldi	r31, 0x06	; 6
     786:	10 82       	st	Z, r1
     788:	31 83       	std	Z+1, r19	; 0x01
     78a:	91 83       	std	Z+1, r25	; 0x01
     78c:	44 e0       	ldi	r20, 0x04	; 4
     78e:	41 83       	std	Z+1, r20	; 0x01
     790:	21 83       	std	Z+1, r18	; 0x01
     792:	80 e1       	ldi	r24, 0x10	; 16
     794:	81 83       	std	Z+1, r24	; 0x01
     796:	80 e2       	ldi	r24, 0x20	; 32
     798:	81 83       	std	Z+1, r24	; 0x01
     79a:	80 e8       	ldi	r24, 0x80	; 128
     79c:	81 83       	std	Z+1, r24	; 0x01
     79e:	81 e1       	ldi	r24, 0x11	; 17
     7a0:	84 83       	std	Z+4, r24	; 0x04
     7a2:	e0 e8       	ldi	r30, 0x80	; 128
     7a4:	f6 e0       	ldi	r31, 0x06	; 6
     7a6:	10 82       	st	Z, r1
     7a8:	31 83       	std	Z+1, r19	; 0x01
     7aa:	91 83       	std	Z+1, r25	; 0x01
     7ac:	41 83       	std	Z+1, r20	; 0x01
     7ae:	21 83       	std	Z+1, r18	; 0x01
     7b0:	14 82       	std	Z+4, r1	; 0x04
     7b2:	08 95       	ret

000007b4 <SetClock>:
     7b4:	8b ec       	ldi	r24, 0xCB	; 203
     7b6:	e0 e5       	ldi	r30, 0x50	; 80
     7b8:	f0 e0       	ldi	r31, 0x00	; 0
     7ba:	82 83       	std	Z+2, r24	; 0x02
     7bc:	80 91 50 00 	lds	r24, 0x0050
     7c0:	88 60       	ori	r24, 0x08	; 8
     7c2:	80 93 50 00 	sts	0x0050, r24
     7c6:	80 91 51 00 	lds	r24, 0x0051
     7ca:	83 ff       	sbrs	r24, 3
     7cc:	fc cf       	rjmp	.-8      	; 0x7c6 <SetClock+0x12>
     7ce:	82 ec       	ldi	r24, 0xC2	; 194
     7d0:	e0 e5       	ldi	r30, 0x50	; 80
     7d2:	f0 e0       	ldi	r31, 0x00	; 0
     7d4:	85 83       	std	Z+5, r24	; 0x05
     7d6:	80 91 50 00 	lds	r24, 0x0050
     7da:	80 61       	ori	r24, 0x10	; 16
     7dc:	80 93 50 00 	sts	0x0050, r24
     7e0:	80 91 51 00 	lds	r24, 0x0051
     7e4:	84 ff       	sbrs	r24, 4
     7e6:	fc cf       	rjmp	.-8      	; 0x7e0 <SetClock+0x2c>
     7e8:	88 ed       	ldi	r24, 0xD8	; 216
     7ea:	84 bf       	out	0x34, r24	; 52
     7ec:	84 e0       	ldi	r24, 0x04	; 4
     7ee:	80 93 40 00 	sts	0x0040, r24
     7f2:	80 91 50 00 	lds	r24, 0x0050
     7f6:	80 93 50 00 	sts	0x0050, r24
     7fa:	08 95       	ret

000007fc <SetTimer>:
     7fc:	e0 e0       	ldi	r30, 0x00	; 0
     7fe:	f8 e0       	ldi	r31, 0x08	; 8
     800:	85 e0       	ldi	r24, 0x05	; 5
     802:	80 83       	st	Z, r24
     804:	81 e1       	ldi	r24, 0x11	; 17
     806:	81 83       	std	Z+1, r24	; 0x01
     808:	12 82       	std	Z+2, r1	; 0x02
     80a:	13 82       	std	Z+3, r1	; 0x03
     80c:	14 82       	std	Z+4, r1	; 0x04
     80e:	88 ee       	ldi	r24, 0xE8	; 232
     810:	93 e0       	ldi	r25, 0x03	; 3
     812:	80 a7       	std	Z+40, r24	; 0x28
     814:	91 a7       	std	Z+41, r25	; 0x29
     816:	83 ef       	ldi	r24, 0xF3	; 243
     818:	84 87       	std	Z+12, r24	; 0x0c
     81a:	16 82       	std	Z+6, r1	; 0x06
     81c:	83 e0       	ldi	r24, 0x03	; 3
     81e:	87 83       	std	Z+7, r24	; 0x07
     820:	08 95       	ret

00000822 <CopyArray>:
     822:	cf 93       	push	r28
     824:	df 93       	push	r29
     826:	fc 01       	movw	r30, r24
     828:	db 01       	movw	r26, r22
     82a:	21 30       	cpi	r18, 0x01	; 1
     82c:	a1 f0       	breq	.+40     	; 0x856 <CopyArray+0x34>
     82e:	21 30       	cpi	r18, 0x01	; 1
     830:	20 f0       	brcs	.+8      	; 0x83a <CopyArray+0x18>
     832:	22 30       	cpi	r18, 0x02	; 2
     834:	09 f0       	breq	.+2      	; 0x838 <CopyArray+0x16>
     836:	6f c0       	rjmp	.+222    	; 0x916 <CopyArray+0xf4>
     838:	59 c0       	rjmp	.+178    	; 0x8ec <CopyArray+0xca>
     83a:	ec 01       	movw	r28, r24
     83c:	20 e0       	ldi	r18, 0x00	; 0
     83e:	30 e0       	ldi	r19, 0x00	; 0
     840:	07 c0       	rjmp	.+14     	; 0x850 <CopyArray+0x2e>
     842:	fd 01       	movw	r30, r26
     844:	e2 0f       	add	r30, r18
     846:	f3 1f       	adc	r31, r19
     848:	89 91       	ld	r24, Y+
     84a:	80 83       	st	Z, r24
     84c:	2f 5f       	subi	r18, 0xFF	; 255
     84e:	3f 4f       	sbci	r19, 0xFF	; 255
     850:	24 17       	cp	r18, r20
     852:	b8 f3       	brcs	.-18     	; 0x842 <CopyArray+0x20>
     854:	60 c0       	rjmp	.+192    	; 0x916 <CopyArray+0xf4>
     856:	91 81       	ldd	r25, Z+1	; 0x01
     858:	96 95       	lsr	r25
     85a:	96 95       	lsr	r25
     85c:	9c 93       	st	X, r25
     85e:	81 81       	ldd	r24, Z+1	; 0x01
     860:	87 ff       	sbrs	r24, 7
     862:	02 c0       	rjmp	.+4      	; 0x868 <CopyArray+0x46>
     864:	90 6c       	ori	r25, 0xC0	; 192
     866:	9c 93       	st	X, r25
     868:	81 81       	ldd	r24, Z+1	; 0x01
     86a:	82 95       	swap	r24
     86c:	88 0f       	add	r24, r24
     86e:	88 0f       	add	r24, r24
     870:	80 7c       	andi	r24, 0xC0	; 192
     872:	90 81       	ld	r25, Z
     874:	96 95       	lsr	r25
     876:	96 95       	lsr	r25
     878:	89 2b       	or	r24, r25
     87a:	11 96       	adiw	r26, 0x01	; 1
     87c:	8c 93       	st	X, r24
     87e:	11 97       	sbiw	r26, 0x01	; 1
     880:	93 81       	ldd	r25, Z+3	; 0x03
     882:	96 95       	lsr	r25
     884:	96 95       	lsr	r25
     886:	12 96       	adiw	r26, 0x02	; 2
     888:	9c 93       	st	X, r25
     88a:	12 97       	sbiw	r26, 0x02	; 2
     88c:	83 81       	ldd	r24, Z+3	; 0x03
     88e:	87 ff       	sbrs	r24, 7
     890:	04 c0       	rjmp	.+8      	; 0x89a <CopyArray+0x78>
     892:	90 6c       	ori	r25, 0xC0	; 192
     894:	12 96       	adiw	r26, 0x02	; 2
     896:	9c 93       	st	X, r25
     898:	12 97       	sbiw	r26, 0x02	; 2
     89a:	83 81       	ldd	r24, Z+3	; 0x03
     89c:	82 95       	swap	r24
     89e:	88 0f       	add	r24, r24
     8a0:	88 0f       	add	r24, r24
     8a2:	80 7c       	andi	r24, 0xC0	; 192
     8a4:	92 81       	ldd	r25, Z+2	; 0x02
     8a6:	96 95       	lsr	r25
     8a8:	96 95       	lsr	r25
     8aa:	89 2b       	or	r24, r25
     8ac:	13 96       	adiw	r26, 0x03	; 3
     8ae:	8c 93       	st	X, r24
     8b0:	13 97       	sbiw	r26, 0x03	; 3
     8b2:	95 81       	ldd	r25, Z+5	; 0x05
     8b4:	96 95       	lsr	r25
     8b6:	96 95       	lsr	r25
     8b8:	14 96       	adiw	r26, 0x04	; 4
     8ba:	9c 93       	st	X, r25
     8bc:	14 97       	sbiw	r26, 0x04	; 4
     8be:	85 81       	ldd	r24, Z+5	; 0x05
     8c0:	87 ff       	sbrs	r24, 7
     8c2:	04 c0       	rjmp	.+8      	; 0x8cc <CopyArray+0xaa>
     8c4:	90 6c       	ori	r25, 0xC0	; 192
     8c6:	14 96       	adiw	r26, 0x04	; 4
     8c8:	9c 93       	st	X, r25
     8ca:	14 97       	sbiw	r26, 0x04	; 4
     8cc:	85 81       	ldd	r24, Z+5	; 0x05
     8ce:	82 95       	swap	r24
     8d0:	88 0f       	add	r24, r24
     8d2:	88 0f       	add	r24, r24
     8d4:	80 7c       	andi	r24, 0xC0	; 192
     8d6:	94 81       	ldd	r25, Z+4	; 0x04
     8d8:	96 95       	lsr	r25
     8da:	96 95       	lsr	r25
     8dc:	89 2b       	or	r24, r25
     8de:	15 96       	adiw	r26, 0x05	; 5
     8e0:	8c 93       	st	X, r24
     8e2:	15 97       	sbiw	r26, 0x05	; 5
     8e4:	86 81       	ldd	r24, Z+6	; 0x06
     8e6:	16 96       	adiw	r26, 0x06	; 6
     8e8:	8c 93       	st	X, r24
     8ea:	15 c0       	rjmp	.+42     	; 0x916 <CopyArray+0xf4>
     8ec:	80 81       	ld	r24, Z
     8ee:	8c 93       	st	X, r24
     8f0:	81 81       	ldd	r24, Z+1	; 0x01
     8f2:	11 96       	adiw	r26, 0x01	; 1
     8f4:	8c 93       	st	X, r24
     8f6:	11 97       	sbiw	r26, 0x01	; 1
     8f8:	84 81       	ldd	r24, Z+4	; 0x04
     8fa:	12 96       	adiw	r26, 0x02	; 2
     8fc:	8c 93       	st	X, r24
     8fe:	12 97       	sbiw	r26, 0x02	; 2
     900:	85 81       	ldd	r24, Z+5	; 0x05
     902:	13 96       	adiw	r26, 0x03	; 3
     904:	8c 93       	st	X, r24
     906:	13 97       	sbiw	r26, 0x03	; 3
     908:	82 81       	ldd	r24, Z+2	; 0x02
     90a:	14 96       	adiw	r26, 0x04	; 4
     90c:	8c 93       	st	X, r24
     90e:	14 97       	sbiw	r26, 0x04	; 4
     910:	83 81       	ldd	r24, Z+3	; 0x03
     912:	15 96       	adiw	r26, 0x05	; 5
     914:	8c 93       	st	X, r24
     916:	df 91       	pop	r29
     918:	cf 91       	pop	r28
     91a:	08 95       	ret

0000091c <itoa_adc>:
     91c:	df 92       	push	r13
     91e:	ef 92       	push	r14
     920:	ff 92       	push	r15
     922:	0f 93       	push	r16
     924:	1f 93       	push	r17
     926:	df 93       	push	r29
     928:	cf 93       	push	r28
     92a:	cd b7       	in	r28, 0x3d	; 61
     92c:	de b7       	in	r29, 0x3e	; 62
     92e:	a0 97       	sbiw	r28, 0x20	; 32
     930:	cd bf       	out	0x3d, r28	; 61
     932:	de bf       	out	0x3e, r29	; 62
     934:	ac 01       	movw	r20, r24
     936:	7b 01       	movw	r14, r22
     938:	d2 2e       	mov	r13, r18
     93a:	1a 82       	std	Y+2, r1	; 0x02
     93c:	90 e3       	ldi	r25, 0x30	; 48
     93e:	08 c0       	rjmp	.+16     	; 0x950 <itoa_adc+0x34>
     940:	8a 81       	ldd	r24, Y+2	; 0x02
     942:	f7 01       	movw	r30, r14
     944:	e8 0f       	add	r30, r24
     946:	f1 1d       	adc	r31, r1
     948:	90 83       	st	Z, r25
     94a:	8a 81       	ldd	r24, Y+2	; 0x02
     94c:	8f 5f       	subi	r24, 0xFF	; 255
     94e:	8a 83       	std	Y+2, r24	; 0x02
     950:	8a 81       	ldd	r24, Y+2	; 0x02
     952:	8d 15       	cp	r24, r13
     954:	a8 f3       	brcs	.-22     	; 0x940 <itoa_adc+0x24>
     956:	8e 01       	movw	r16, r28
     958:	0d 5f       	subi	r16, 0xFD	; 253
     95a:	1f 4f       	sbci	r17, 0xFF	; 255
     95c:	ca 01       	movw	r24, r20
     95e:	b8 01       	movw	r22, r16
     960:	40 e1       	ldi	r20, 0x10	; 16
     962:	50 e0       	ldi	r21, 0x00	; 0
     964:	0e 94 bc 09 	call	0x1378	; 0x1378 <itoa>
     968:	19 82       	std	Y+1, r1	; 0x01
     96a:	98 01       	movw	r18, r16
     96c:	0a c0       	rjmp	.+20     	; 0x982 <itoa_adc+0x66>
     96e:	89 81       	ldd	r24, Y+1	; 0x01
     970:	f9 01       	movw	r30, r18
     972:	e8 0f       	add	r30, r24
     974:	f1 1d       	adc	r31, r1
     976:	80 81       	ld	r24, Z
     978:	88 23       	and	r24, r24
     97a:	31 f0       	breq	.+12     	; 0x988 <itoa_adc+0x6c>
     97c:	89 81       	ldd	r24, Y+1	; 0x01
     97e:	8f 5f       	subi	r24, 0xFF	; 255
     980:	89 83       	std	Y+1, r24	; 0x01
     982:	89 81       	ldd	r24, Y+1	; 0x01
     984:	8d 31       	cpi	r24, 0x1D	; 29
     986:	98 f3       	brcs	.-26     	; 0x96e <itoa_adc+0x52>
     988:	89 81       	ldd	r24, Y+1	; 0x01
     98a:	d8 16       	cp	r13, r24
     98c:	c8 f0       	brcs	.+50     	; 0x9c0 <itoa_adc+0xa4>
     98e:	89 81       	ldd	r24, Y+1	; 0x01
     990:	88 23       	and	r24, r24
     992:	b1 f0       	breq	.+44     	; 0x9c0 <itoa_adc+0xa4>
     994:	89 81       	ldd	r24, Y+1	; 0x01
     996:	8a 83       	std	Y+2, r24	; 0x02
     998:	9e 01       	movw	r18, r28
     99a:	2d 5f       	subi	r18, 0xFD	; 253
     99c:	3f 4f       	sbci	r19, 0xFF	; 255
     99e:	0d c0       	rjmp	.+26     	; 0x9ba <itoa_adc+0x9e>
     9a0:	8a 81       	ldd	r24, Y+2	; 0x02
     9a2:	9a 81       	ldd	r25, Y+2	; 0x02
     9a4:	d7 01       	movw	r26, r14
     9a6:	a8 0f       	add	r26, r24
     9a8:	b1 1d       	adc	r27, r1
     9aa:	f9 01       	movw	r30, r18
     9ac:	e9 0f       	add	r30, r25
     9ae:	f1 1d       	adc	r31, r1
     9b0:	80 81       	ld	r24, Z
     9b2:	8c 93       	st	X, r24
     9b4:	8a 81       	ldd	r24, Y+2	; 0x02
     9b6:	81 50       	subi	r24, 0x01	; 1
     9b8:	8a 83       	std	Y+2, r24	; 0x02
     9ba:	8a 81       	ldd	r24, Y+2	; 0x02
     9bc:	88 23       	and	r24, r24
     9be:	81 f7       	brne	.-32     	; 0x9a0 <itoa_adc+0x84>
     9c0:	a0 96       	adiw	r28, 0x20	; 32
     9c2:	cd bf       	out	0x3d, r28	; 61
     9c4:	de bf       	out	0x3e, r29	; 62
     9c6:	cf 91       	pop	r28
     9c8:	df 91       	pop	r29
     9ca:	1f 91       	pop	r17
     9cc:	0f 91       	pop	r16
     9ce:	ff 90       	pop	r15
     9d0:	ef 90       	pop	r14
     9d2:	df 90       	pop	r13
     9d4:	08 95       	ret

000009d6 <TerminalShowInfo>:
     9d6:	60 e0       	ldi	r22, 0x00	; 0
     9d8:	01 c0       	rjmp	.+2      	; 0x9dc <TerminalShowInfo+0x6>
     9da:	6f 5f       	subi	r22, 0xFF	; 255
     9dc:	e6 2f       	mov	r30, r22
     9de:	f0 e0       	ldi	r31, 0x00	; 0
     9e0:	ec 5c       	subi	r30, 0xCC	; 204
     9e2:	ff 4d       	sbci	r31, 0xDF	; 223
     9e4:	80 81       	ld	r24, Z
     9e6:	88 23       	and	r24, r24
     9e8:	c1 f7       	brne	.-16     	; 0x9da <TerminalShowInfo+0x4>
     9ea:	84 e3       	ldi	r24, 0x34	; 52
     9ec:	90 e2       	ldi	r25, 0x20	; 32
     9ee:	0e 94 e0 02 	call	0x5c0	; 0x5c0 <USBUartSendArray>
     9f2:	08 95       	ret

000009f4 <TerminalCommandsNoArgument>:
     9f4:	1f 93       	push	r17
     9f6:	fc 01       	movw	r30, r24
     9f8:	80 81       	ld	r24, Z
     9fa:	81 36       	cpi	r24, 0x61	; 97
     9fc:	09 f4       	brne	.+2      	; 0xa00 <TerminalCommandsNoArgument+0xc>
     9fe:	63 c0       	rjmp	.+198    	; 0xac6 <TerminalCommandsNoArgument+0xd2>
     a00:	84 36       	cpi	r24, 0x64	; 100
     a02:	51 f0       	breq	.+20     	; 0xa18 <TerminalCommandsNoArgument+0x24>
     a04:	8f 33       	cpi	r24, 0x3F	; 63
     a06:	09 f0       	breq	.+2      	; 0xa0a <TerminalCommandsNoArgument+0x16>
     a08:	26 c1       	rjmp	.+588    	; 0xc56 <TerminalCommandsNoArgument+0x262>
     a0a:	81 81       	ldd	r24, Z+1	; 0x01
     a0c:	8f 33       	cpi	r24, 0x3F	; 63
     a0e:	09 f0       	breq	.+2      	; 0xa12 <TerminalCommandsNoArgument+0x1e>
     a10:	22 c1       	rjmp	.+580    	; 0xc56 <TerminalCommandsNoArgument+0x262>
     a12:	0e 94 eb 04 	call	0x9d6	; 0x9d6 <TerminalShowInfo>
     a16:	a1 c0       	rjmp	.+322    	; 0xb5a <TerminalCommandsNoArgument+0x166>
     a18:	8b e3       	ldi	r24, 0x3B	; 59
     a1a:	80 93 ed 20 	sts	0x20ED, r24
     a1e:	80 e3       	ldi	r24, 0x30	; 48
     a20:	80 93 ee 20 	sts	0x20EE, r24
     a24:	88 e7       	ldi	r24, 0x78	; 120
     a26:	80 93 ef 20 	sts	0x20EF, r24
     a2a:	80 e2       	ldi	r24, 0x20	; 32
     a2c:	80 93 f0 20 	sts	0x20F0, r24
     a30:	80 93 f1 20 	sts	0x20F1, r24
     a34:	80 93 f2 20 	sts	0x20F2, r24
     a38:	80 93 f3 20 	sts	0x20F3, r24
     a3c:	80 93 f4 20 	sts	0x20F4, r24
     a40:	80 93 f5 20 	sts	0x20F5, r24
     a44:	80 91 24 20 	lds	r24, 0x2024
     a48:	80 93 f6 20 	sts	0x20F6, r24
     a4c:	80 91 25 20 	lds	r24, 0x2025
     a50:	80 93 f7 20 	sts	0x20F7, r24
     a54:	80 91 26 20 	lds	r24, 0x2026
     a58:	80 93 f8 20 	sts	0x20F8, r24
     a5c:	80 91 27 20 	lds	r24, 0x2027
     a60:	80 93 f9 20 	sts	0x20F9, r24
     a64:	81 81       	ldd	r24, Z+1	; 0x01
     a66:	82 33       	cpi	r24, 0x32	; 50
     a68:	d1 f0       	breq	.+52     	; 0xa9e <TerminalCommandsNoArgument+0xaa>
     a6a:	83 33       	cpi	r24, 0x33	; 51
     a6c:	30 f4       	brcc	.+12     	; 0xa7a <TerminalCommandsNoArgument+0x86>
     a6e:	80 33       	cpi	r24, 0x30	; 48
     a70:	61 f0       	breq	.+24     	; 0xa8a <TerminalCommandsNoArgument+0x96>
     a72:	81 33       	cpi	r24, 0x31	; 49
     a74:	09 f0       	breq	.+2      	; 0xa78 <TerminalCommandsNoArgument+0x84>
     a76:	ef c0       	rjmp	.+478    	; 0xc56 <TerminalCommandsNoArgument+0x262>
     a78:	0d c0       	rjmp	.+26     	; 0xa94 <TerminalCommandsNoArgument+0xa0>
     a7a:	84 33       	cpi	r24, 0x34	; 52
     a7c:	d1 f0       	breq	.+52     	; 0xab2 <TerminalCommandsNoArgument+0xbe>
     a7e:	84 33       	cpi	r24, 0x34	; 52
     a80:	98 f0       	brcs	.+38     	; 0xaa8 <TerminalCommandsNoArgument+0xb4>
     a82:	85 33       	cpi	r24, 0x35	; 53
     a84:	09 f0       	breq	.+2      	; 0xa88 <TerminalCommandsNoArgument+0x94>
     a86:	e7 c0       	rjmp	.+462    	; 0xc56 <TerminalCommandsNoArgument+0x262>
     a88:	19 c0       	rjmp	.+50     	; 0xabc <TerminalCommandsNoArgument+0xc8>
     a8a:	80 91 28 20 	lds	r24, 0x2028
     a8e:	90 91 29 20 	lds	r25, 0x2029
     a92:	58 c0       	rjmp	.+176    	; 0xb44 <TerminalCommandsNoArgument+0x150>
     a94:	80 91 2a 20 	lds	r24, 0x202A
     a98:	90 91 2b 20 	lds	r25, 0x202B
     a9c:	53 c0       	rjmp	.+166    	; 0xb44 <TerminalCommandsNoArgument+0x150>
     a9e:	80 91 2c 20 	lds	r24, 0x202C
     aa2:	90 91 2d 20 	lds	r25, 0x202D
     aa6:	4e c0       	rjmp	.+156    	; 0xb44 <TerminalCommandsNoArgument+0x150>
     aa8:	80 91 2e 20 	lds	r24, 0x202E
     aac:	90 91 2f 20 	lds	r25, 0x202F
     ab0:	49 c0       	rjmp	.+146    	; 0xb44 <TerminalCommandsNoArgument+0x150>
     ab2:	80 91 30 20 	lds	r24, 0x2030
     ab6:	90 91 31 20 	lds	r25, 0x2031
     aba:	44 c0       	rjmp	.+136    	; 0xb44 <TerminalCommandsNoArgument+0x150>
     abc:	80 91 32 20 	lds	r24, 0x2032
     ac0:	90 91 33 20 	lds	r25, 0x2033
     ac4:	3f c0       	rjmp	.+126    	; 0xb44 <TerminalCommandsNoArgument+0x150>
     ac6:	8b e3       	ldi	r24, 0x3B	; 59
     ac8:	80 93 ed 20 	sts	0x20ED, r24
     acc:	80 e3       	ldi	r24, 0x30	; 48
     ace:	80 93 ee 20 	sts	0x20EE, r24
     ad2:	88 e7       	ldi	r24, 0x78	; 120
     ad4:	80 93 ef 20 	sts	0x20EF, r24
     ad8:	80 e2       	ldi	r24, 0x20	; 32
     ada:	80 93 f0 20 	sts	0x20F0, r24
     ade:	80 93 f1 20 	sts	0x20F1, r24
     ae2:	80 93 f2 20 	sts	0x20F2, r24
     ae6:	80 93 f3 20 	sts	0x20F3, r24
     aea:	80 93 f4 20 	sts	0x20F4, r24
     aee:	80 93 f5 20 	sts	0x20F5, r24
     af2:	80 91 24 20 	lds	r24, 0x2024
     af6:	80 93 f6 20 	sts	0x20F6, r24
     afa:	80 91 25 20 	lds	r24, 0x2025
     afe:	80 93 f7 20 	sts	0x20F7, r24
     b02:	80 91 26 20 	lds	r24, 0x2026
     b06:	80 93 f8 20 	sts	0x20F8, r24
     b0a:	80 91 27 20 	lds	r24, 0x2027
     b0e:	80 93 f9 20 	sts	0x20F9, r24
     b12:	81 81       	ldd	r24, Z+1	; 0x01
     b14:	82 33       	cpi	r24, 0x32	; 50
     b16:	41 f1       	breq	.+80     	; 0xb68 <TerminalCommandsNoArgument+0x174>
     b18:	83 33       	cpi	r24, 0x33	; 51
     b1a:	40 f4       	brcc	.+16     	; 0xb2c <TerminalCommandsNoArgument+0x138>
     b1c:	80 33       	cpi	r24, 0x30	; 48
     b1e:	71 f0       	breq	.+28     	; 0xb3c <TerminalCommandsNoArgument+0x148>
     b20:	81 33       	cpi	r24, 0x31	; 49
     b22:	e8 f4       	brcc	.+58     	; 0xb5e <TerminalCommandsNoArgument+0x16a>
     b24:	8a 32       	cpi	r24, 0x2A	; 42
     b26:	09 f0       	breq	.+2      	; 0xb2a <TerminalCommandsNoArgument+0x136>
     b28:	96 c0       	rjmp	.+300    	; 0xc56 <TerminalCommandsNoArgument+0x262>
     b2a:	35 c0       	rjmp	.+106    	; 0xb96 <TerminalCommandsNoArgument+0x1a2>
     b2c:	84 33       	cpi	r24, 0x34	; 52
     b2e:	31 f1       	breq	.+76     	; 0xb7c <TerminalCommandsNoArgument+0x188>
     b30:	84 33       	cpi	r24, 0x34	; 52
     b32:	f8 f0       	brcs	.+62     	; 0xb72 <TerminalCommandsNoArgument+0x17e>
     b34:	85 33       	cpi	r24, 0x35	; 53
     b36:	09 f0       	breq	.+2      	; 0xb3a <TerminalCommandsNoArgument+0x146>
     b38:	8e c0       	rjmp	.+284    	; 0xc56 <TerminalCommandsNoArgument+0x262>
     b3a:	25 c0       	rjmp	.+74     	; 0xb86 <TerminalCommandsNoArgument+0x192>
     b3c:	80 91 d4 22 	lds	r24, 0x22D4
     b40:	90 91 d5 22 	lds	r25, 0x22D5
     b44:	60 ef       	ldi	r22, 0xF0	; 240
     b46:	70 e2       	ldi	r23, 0x20	; 32
     b48:	40 e1       	ldi	r20, 0x10	; 16
     b4a:	50 e0       	ldi	r21, 0x00	; 0
     b4c:	0e 94 bc 09 	call	0x1378	; 0x1378 <itoa>
     b50:	8d ee       	ldi	r24, 0xED	; 237
     b52:	90 e2       	ldi	r25, 0x20	; 32
     b54:	6d e0       	ldi	r22, 0x0D	; 13
     b56:	0e 94 e0 02 	call	0x5c0	; 0x5c0 <USBUartSendArray>
     b5a:	80 e0       	ldi	r24, 0x00	; 0
     b5c:	7d c0       	rjmp	.+250    	; 0xc58 <TerminalCommandsNoArgument+0x264>
     b5e:	80 91 d6 22 	lds	r24, 0x22D6
     b62:	90 91 d7 22 	lds	r25, 0x22D7
     b66:	ee cf       	rjmp	.-36     	; 0xb44 <TerminalCommandsNoArgument+0x150>
     b68:	80 91 d8 22 	lds	r24, 0x22D8
     b6c:	90 91 d9 22 	lds	r25, 0x22D9
     b70:	e9 cf       	rjmp	.-46     	; 0xb44 <TerminalCommandsNoArgument+0x150>
     b72:	80 91 da 22 	lds	r24, 0x22DA
     b76:	90 91 db 22 	lds	r25, 0x22DB
     b7a:	e4 cf       	rjmp	.-56     	; 0xb44 <TerminalCommandsNoArgument+0x150>
     b7c:	80 91 dc 22 	lds	r24, 0x22DC
     b80:	90 91 dd 22 	lds	r25, 0x22DD
     b84:	df cf       	rjmp	.-66     	; 0xb44 <TerminalCommandsNoArgument+0x150>
     b86:	80 91 de 22 	lds	r24, 0x22DE
     b8a:	90 91 df 22 	lds	r25, 0x22DF
     b8e:	da cf       	rjmp	.-76     	; 0xb44 <TerminalCommandsNoArgument+0x150>
     b90:	10 93 ed 20 	sts	0x20ED, r17
     b94:	01 c0       	rjmp	.+2      	; 0xb98 <TerminalCommandsNoArgument+0x1a4>
     b96:	1a e0       	ldi	r17, 0x0A	; 10
     b98:	0e 94 91 01 	call	0x322	; 0x322 <SPIBufferAvailable>
     b9c:	88 23       	and	r24, r24
     b9e:	c1 f3       	breq	.-16     	; 0xb90 <TerminalCommandsNoArgument+0x19c>
     ba0:	80 91 d4 22 	lds	r24, 0x22D4
     ba4:	90 91 d5 22 	lds	r25, 0x22D5
     ba8:	6e ee       	ldi	r22, 0xEE	; 238
     baa:	70 e2       	ldi	r23, 0x20	; 32
     bac:	40 e1       	ldi	r20, 0x10	; 16
     bae:	24 e0       	ldi	r18, 0x04	; 4
     bb0:	0e 94 8e 04 	call	0x91c	; 0x91c <itoa_adc>
     bb4:	10 e2       	ldi	r17, 0x20	; 32
     bb6:	10 93 f2 20 	sts	0x20F2, r17
     bba:	80 91 d6 22 	lds	r24, 0x22D6
     bbe:	90 91 d7 22 	lds	r25, 0x22D7
     bc2:	63 ef       	ldi	r22, 0xF3	; 243
     bc4:	70 e2       	ldi	r23, 0x20	; 32
     bc6:	40 e1       	ldi	r20, 0x10	; 16
     bc8:	24 e0       	ldi	r18, 0x04	; 4
     bca:	0e 94 8e 04 	call	0x91c	; 0x91c <itoa_adc>
     bce:	10 93 f7 20 	sts	0x20F7, r17
     bd2:	80 91 d8 22 	lds	r24, 0x22D8
     bd6:	90 91 d9 22 	lds	r25, 0x22D9
     bda:	68 ef       	ldi	r22, 0xF8	; 248
     bdc:	70 e2       	ldi	r23, 0x20	; 32
     bde:	40 e1       	ldi	r20, 0x10	; 16
     be0:	24 e0       	ldi	r18, 0x04	; 4
     be2:	0e 94 8e 04 	call	0x91c	; 0x91c <itoa_adc>
     be6:	10 93 fc 20 	sts	0x20FC, r17
     bea:	80 91 da 22 	lds	r24, 0x22DA
     bee:	90 91 db 22 	lds	r25, 0x22DB
     bf2:	6d ef       	ldi	r22, 0xFD	; 253
     bf4:	70 e2       	ldi	r23, 0x20	; 32
     bf6:	40 e1       	ldi	r20, 0x10	; 16
     bf8:	24 e0       	ldi	r18, 0x04	; 4
     bfa:	0e 94 8e 04 	call	0x91c	; 0x91c <itoa_adc>
     bfe:	10 93 01 21 	sts	0x2101, r17
     c02:	80 91 dc 22 	lds	r24, 0x22DC
     c06:	90 91 dd 22 	lds	r25, 0x22DD
     c0a:	62 e0       	ldi	r22, 0x02	; 2
     c0c:	71 e2       	ldi	r23, 0x21	; 33
     c0e:	40 e1       	ldi	r20, 0x10	; 16
     c10:	24 e0       	ldi	r18, 0x04	; 4
     c12:	0e 94 8e 04 	call	0x91c	; 0x91c <itoa_adc>
     c16:	10 93 06 21 	sts	0x2106, r17
     c1a:	80 91 de 22 	lds	r24, 0x22DE
     c1e:	90 91 df 22 	lds	r25, 0x22DF
     c22:	67 e0       	ldi	r22, 0x07	; 7
     c24:	71 e2       	ldi	r23, 0x21	; 33
     c26:	40 e1       	ldi	r20, 0x10	; 16
     c28:	24 e0       	ldi	r18, 0x04	; 4
     c2a:	0e 94 8e 04 	call	0x91c	; 0x91c <itoa_adc>
     c2e:	80 91 24 20 	lds	r24, 0x2024
     c32:	80 93 0b 21 	sts	0x210B, r24
     c36:	80 91 25 20 	lds	r24, 0x2025
     c3a:	80 93 0c 21 	sts	0x210C, r24
     c3e:	80 91 26 20 	lds	r24, 0x2026
     c42:	80 93 0d 21 	sts	0x210D, r24
     c46:	80 91 27 20 	lds	r24, 0x2027
     c4a:	80 93 0e 21 	sts	0x210E, r24
     c4e:	8d ee       	ldi	r24, 0xED	; 237
     c50:	90 e2       	ldi	r25, 0x20	; 32
     c52:	62 e2       	ldi	r22, 0x22	; 34
     c54:	80 cf       	rjmp	.-256    	; 0xb56 <TerminalCommandsNoArgument+0x162>
     c56:	81 e0       	ldi	r24, 0x01	; 1
     c58:	1f 91       	pop	r17
     c5a:	08 95       	ret

00000c5c <TerminalCommandsWithArgument>:
     c5c:	ef 92       	push	r14
     c5e:	ff 92       	push	r15
     c60:	0f 93       	push	r16
     c62:	1f 93       	push	r17
     c64:	fc 01       	movw	r30, r24
     c66:	80 81       	ld	r24, Z
     c68:	84 36       	cpi	r24, 0x64	; 100
     c6a:	09 f0       	breq	.+2      	; 0xc6e <TerminalCommandsWithArgument+0x12>
     c6c:	42 c1       	rjmp	.+644    	; 0xef2 <TerminalCommandsWithArgument+0x296>
     c6e:	8b e3       	ldi	r24, 0x3B	; 59
     c70:	80 93 10 21 	sts	0x2110, r24
     c74:	90 e2       	ldi	r25, 0x20	; 32
     c76:	90 93 11 21 	sts	0x2111, r25
     c7a:	90 93 12 21 	sts	0x2112, r25
     c7e:	90 93 13 21 	sts	0x2113, r25
     c82:	90 93 14 21 	sts	0x2114, r25
     c86:	90 93 15 21 	sts	0x2115, r25
     c8a:	90 93 16 21 	sts	0x2116, r25
     c8e:	90 93 17 21 	sts	0x2117, r25
     c92:	90 93 18 21 	sts	0x2118, r25
     c96:	80 91 24 20 	lds	r24, 0x2024
     c9a:	80 93 19 21 	sts	0x2119, r24
     c9e:	80 91 25 20 	lds	r24, 0x2025
     ca2:	80 93 1a 21 	sts	0x211A, r24
     ca6:	80 91 26 20 	lds	r24, 0x2026
     caa:	80 93 1b 21 	sts	0x211B, r24
     cae:	80 91 27 20 	lds	r24, 0x2027
     cb2:	80 93 1c 21 	sts	0x211C, r24
     cb6:	81 81       	ldd	r24, Z+1	; 0x01
     cb8:	82 33       	cpi	r24, 0x32	; 50
     cba:	09 f4       	brne	.+2      	; 0xcbe <TerminalCommandsWithArgument+0x62>
     cbc:	6a c0       	rjmp	.+212    	; 0xd92 <TerminalCommandsWithArgument+0x136>
     cbe:	83 33       	cpi	r24, 0x33	; 51
     cc0:	30 f4       	brcc	.+12     	; 0xcce <TerminalCommandsWithArgument+0x72>
     cc2:	80 33       	cpi	r24, 0x30	; 48
     cc4:	71 f0       	breq	.+28     	; 0xce2 <TerminalCommandsWithArgument+0x86>
     cc6:	81 33       	cpi	r24, 0x31	; 49
     cc8:	09 f0       	breq	.+2      	; 0xccc <TerminalCommandsWithArgument+0x70>
     cca:	13 c1       	rjmp	.+550    	; 0xef2 <TerminalCommandsWithArgument+0x296>
     ccc:	36 c0       	rjmp	.+108    	; 0xd3a <TerminalCommandsWithArgument+0xde>
     cce:	84 33       	cpi	r24, 0x34	; 52
     cd0:	09 f4       	brne	.+2      	; 0xcd4 <TerminalCommandsWithArgument+0x78>
     cd2:	b7 c0       	rjmp	.+366    	; 0xe42 <TerminalCommandsWithArgument+0x1e6>
     cd4:	84 33       	cpi	r24, 0x34	; 52
     cd6:	08 f4       	brcc	.+2      	; 0xcda <TerminalCommandsWithArgument+0x7e>
     cd8:	88 c0       	rjmp	.+272    	; 0xdea <TerminalCommandsWithArgument+0x18e>
     cda:	85 33       	cpi	r24, 0x35	; 53
     cdc:	09 f0       	breq	.+2      	; 0xce0 <TerminalCommandsWithArgument+0x84>
     cde:	09 c1       	rjmp	.+530    	; 0xef2 <TerminalCommandsWithArgument+0x296>
     ce0:	dd c0       	rjmp	.+442    	; 0xe9c <TerminalCommandsWithArgument+0x240>
     ce2:	fa 01       	movw	r30, r20
     ce4:	e6 0f       	add	r30, r22
     ce6:	f1 1d       	adc	r31, r1
     ce8:	90 83       	st	Z, r25
     cea:	ca 01       	movw	r24, r20
     cec:	60 e0       	ldi	r22, 0x00	; 0
     cee:	70 e0       	ldi	r23, 0x00	; 0
     cf0:	40 e1       	ldi	r20, 0x10	; 16
     cf2:	50 e0       	ldi	r21, 0x00	; 0
     cf4:	0e 94 9e 08 	call	0x113c	; 0x113c <strtoul>
     cf8:	7b 01       	movw	r14, r22
     cfa:	8c 01       	movw	r16, r24
     cfc:	80 e0       	ldi	r24, 0x00	; 0
     cfe:	e8 16       	cp	r14, r24
     d00:	80 e1       	ldi	r24, 0x10	; 16
     d02:	f8 06       	cpc	r15, r24
     d04:	80 e0       	ldi	r24, 0x00	; 0
     d06:	08 07       	cpc	r16, r24
     d08:	80 e0       	ldi	r24, 0x00	; 0
     d0a:	18 07       	cpc	r17, r24
     d0c:	08 f0       	brcs	.+2      	; 0xd10 <TerminalCommandsWithArgument+0xb4>
     d0e:	f1 c0       	rjmp	.+482    	; 0xef2 <TerminalCommandsWithArgument+0x296>
     d10:	c7 01       	movw	r24, r14
     d12:	61 e1       	ldi	r22, 0x11	; 17
     d14:	71 e2       	ldi	r23, 0x21	; 33
     d16:	40 e1       	ldi	r20, 0x10	; 16
     d18:	50 e0       	ldi	r21, 0x00	; 0
     d1a:	0e 94 bc 09 	call	0x1378	; 0x1378 <itoa>
     d1e:	80 e1       	ldi	r24, 0x10	; 16
     d20:	91 e2       	ldi	r25, 0x21	; 33
     d22:	6d e0       	ldi	r22, 0x0D	; 13
     d24:	0e 94 e0 02 	call	0x5c0	; 0x5c0 <USBUartSendArray>
     d28:	c7 01       	movw	r24, r14
     d2a:	60 e0       	ldi	r22, 0x00	; 0
     d2c:	0e 94 45 02 	call	0x48a	; 0x48a <DAC_2636WriteSingleChannel>
     d30:	e0 92 28 20 	sts	0x2028, r14
     d34:	f0 92 29 20 	sts	0x2029, r15
     d38:	af c0       	rjmp	.+350    	; 0xe98 <TerminalCommandsWithArgument+0x23c>
     d3a:	fa 01       	movw	r30, r20
     d3c:	e6 0f       	add	r30, r22
     d3e:	f1 1d       	adc	r31, r1
     d40:	90 83       	st	Z, r25
     d42:	ca 01       	movw	r24, r20
     d44:	60 e0       	ldi	r22, 0x00	; 0
     d46:	70 e0       	ldi	r23, 0x00	; 0
     d48:	40 e1       	ldi	r20, 0x10	; 16
     d4a:	50 e0       	ldi	r21, 0x00	; 0
     d4c:	0e 94 9e 08 	call	0x113c	; 0x113c <strtoul>
     d50:	7b 01       	movw	r14, r22
     d52:	8c 01       	movw	r16, r24
     d54:	80 e0       	ldi	r24, 0x00	; 0
     d56:	e8 16       	cp	r14, r24
     d58:	80 e1       	ldi	r24, 0x10	; 16
     d5a:	f8 06       	cpc	r15, r24
     d5c:	80 e0       	ldi	r24, 0x00	; 0
     d5e:	08 07       	cpc	r16, r24
     d60:	80 e0       	ldi	r24, 0x00	; 0
     d62:	18 07       	cpc	r17, r24
     d64:	08 f0       	brcs	.+2      	; 0xd68 <TerminalCommandsWithArgument+0x10c>
     d66:	c5 c0       	rjmp	.+394    	; 0xef2 <TerminalCommandsWithArgument+0x296>
     d68:	c7 01       	movw	r24, r14
     d6a:	61 e1       	ldi	r22, 0x11	; 17
     d6c:	71 e2       	ldi	r23, 0x21	; 33
     d6e:	40 e1       	ldi	r20, 0x10	; 16
     d70:	50 e0       	ldi	r21, 0x00	; 0
     d72:	0e 94 bc 09 	call	0x1378	; 0x1378 <itoa>
     d76:	80 e1       	ldi	r24, 0x10	; 16
     d78:	91 e2       	ldi	r25, 0x21	; 33
     d7a:	6d e0       	ldi	r22, 0x0D	; 13
     d7c:	0e 94 e0 02 	call	0x5c0	; 0x5c0 <USBUartSendArray>
     d80:	c7 01       	movw	r24, r14
     d82:	61 e0       	ldi	r22, 0x01	; 1
     d84:	0e 94 45 02 	call	0x48a	; 0x48a <DAC_2636WriteSingleChannel>
     d88:	e0 92 2a 20 	sts	0x202A, r14
     d8c:	f0 92 2b 20 	sts	0x202B, r15
     d90:	83 c0       	rjmp	.+262    	; 0xe98 <TerminalCommandsWithArgument+0x23c>
     d92:	fa 01       	movw	r30, r20
     d94:	e6 0f       	add	r30, r22
     d96:	f1 1d       	adc	r31, r1
     d98:	90 83       	st	Z, r25
     d9a:	ca 01       	movw	r24, r20
     d9c:	60 e0       	ldi	r22, 0x00	; 0
     d9e:	70 e0       	ldi	r23, 0x00	; 0
     da0:	40 e1       	ldi	r20, 0x10	; 16
     da2:	50 e0       	ldi	r21, 0x00	; 0
     da4:	0e 94 9e 08 	call	0x113c	; 0x113c <strtoul>
     da8:	7b 01       	movw	r14, r22
     daa:	8c 01       	movw	r16, r24
     dac:	80 e0       	ldi	r24, 0x00	; 0
     dae:	e8 16       	cp	r14, r24
     db0:	80 e1       	ldi	r24, 0x10	; 16
     db2:	f8 06       	cpc	r15, r24
     db4:	80 e0       	ldi	r24, 0x00	; 0
     db6:	08 07       	cpc	r16, r24
     db8:	80 e0       	ldi	r24, 0x00	; 0
     dba:	18 07       	cpc	r17, r24
     dbc:	08 f0       	brcs	.+2      	; 0xdc0 <TerminalCommandsWithArgument+0x164>
     dbe:	99 c0       	rjmp	.+306    	; 0xef2 <TerminalCommandsWithArgument+0x296>
     dc0:	c7 01       	movw	r24, r14
     dc2:	61 e1       	ldi	r22, 0x11	; 17
     dc4:	71 e2       	ldi	r23, 0x21	; 33
     dc6:	40 e1       	ldi	r20, 0x10	; 16
     dc8:	50 e0       	ldi	r21, 0x00	; 0
     dca:	0e 94 bc 09 	call	0x1378	; 0x1378 <itoa>
     dce:	80 e1       	ldi	r24, 0x10	; 16
     dd0:	91 e2       	ldi	r25, 0x21	; 33
     dd2:	6d e0       	ldi	r22, 0x0D	; 13
     dd4:	0e 94 e0 02 	call	0x5c0	; 0x5c0 <USBUartSendArray>
     dd8:	c7 01       	movw	r24, r14
     dda:	62 e0       	ldi	r22, 0x02	; 2
     ddc:	0e 94 45 02 	call	0x48a	; 0x48a <DAC_2636WriteSingleChannel>
     de0:	e0 92 2c 20 	sts	0x202C, r14
     de4:	f0 92 2d 20 	sts	0x202D, r15
     de8:	57 c0       	rjmp	.+174    	; 0xe98 <TerminalCommandsWithArgument+0x23c>
     dea:	fa 01       	movw	r30, r20
     dec:	e6 0f       	add	r30, r22
     dee:	f1 1d       	adc	r31, r1
     df0:	90 83       	st	Z, r25
     df2:	ca 01       	movw	r24, r20
     df4:	60 e0       	ldi	r22, 0x00	; 0
     df6:	70 e0       	ldi	r23, 0x00	; 0
     df8:	40 e1       	ldi	r20, 0x10	; 16
     dfa:	50 e0       	ldi	r21, 0x00	; 0
     dfc:	0e 94 9e 08 	call	0x113c	; 0x113c <strtoul>
     e00:	7b 01       	movw	r14, r22
     e02:	8c 01       	movw	r16, r24
     e04:	80 e0       	ldi	r24, 0x00	; 0
     e06:	e8 16       	cp	r14, r24
     e08:	80 e1       	ldi	r24, 0x10	; 16
     e0a:	f8 06       	cpc	r15, r24
     e0c:	80 e0       	ldi	r24, 0x00	; 0
     e0e:	08 07       	cpc	r16, r24
     e10:	80 e0       	ldi	r24, 0x00	; 0
     e12:	18 07       	cpc	r17, r24
     e14:	08 f0       	brcs	.+2      	; 0xe18 <TerminalCommandsWithArgument+0x1bc>
     e16:	6d c0       	rjmp	.+218    	; 0xef2 <TerminalCommandsWithArgument+0x296>
     e18:	c7 01       	movw	r24, r14
     e1a:	61 e1       	ldi	r22, 0x11	; 17
     e1c:	71 e2       	ldi	r23, 0x21	; 33
     e1e:	40 e1       	ldi	r20, 0x10	; 16
     e20:	50 e0       	ldi	r21, 0x00	; 0
     e22:	0e 94 bc 09 	call	0x1378	; 0x1378 <itoa>
     e26:	80 e1       	ldi	r24, 0x10	; 16
     e28:	91 e2       	ldi	r25, 0x21	; 33
     e2a:	6d e0       	ldi	r22, 0x0D	; 13
     e2c:	0e 94 e0 02 	call	0x5c0	; 0x5c0 <USBUartSendArray>
     e30:	c7 01       	movw	r24, r14
     e32:	63 e0       	ldi	r22, 0x03	; 3
     e34:	0e 94 45 02 	call	0x48a	; 0x48a <DAC_2636WriteSingleChannel>
     e38:	e0 92 2e 20 	sts	0x202E, r14
     e3c:	f0 92 2f 20 	sts	0x202F, r15
     e40:	2b c0       	rjmp	.+86     	; 0xe98 <TerminalCommandsWithArgument+0x23c>
     e42:	fa 01       	movw	r30, r20
     e44:	e6 0f       	add	r30, r22
     e46:	f1 1d       	adc	r31, r1
     e48:	90 83       	st	Z, r25
     e4a:	ca 01       	movw	r24, r20
     e4c:	60 e0       	ldi	r22, 0x00	; 0
     e4e:	70 e0       	ldi	r23, 0x00	; 0
     e50:	40 e1       	ldi	r20, 0x10	; 16
     e52:	50 e0       	ldi	r21, 0x00	; 0
     e54:	0e 94 9e 08 	call	0x113c	; 0x113c <strtoul>
     e58:	7b 01       	movw	r14, r22
     e5a:	8c 01       	movw	r16, r24
     e5c:	80 e0       	ldi	r24, 0x00	; 0
     e5e:	e8 16       	cp	r14, r24
     e60:	80 e1       	ldi	r24, 0x10	; 16
     e62:	f8 06       	cpc	r15, r24
     e64:	80 e0       	ldi	r24, 0x00	; 0
     e66:	08 07       	cpc	r16, r24
     e68:	80 e0       	ldi	r24, 0x00	; 0
     e6a:	18 07       	cpc	r17, r24
     e6c:	08 f0       	brcs	.+2      	; 0xe70 <TerminalCommandsWithArgument+0x214>
     e6e:	41 c0       	rjmp	.+130    	; 0xef2 <TerminalCommandsWithArgument+0x296>
     e70:	c7 01       	movw	r24, r14
     e72:	61 e1       	ldi	r22, 0x11	; 17
     e74:	71 e2       	ldi	r23, 0x21	; 33
     e76:	40 e1       	ldi	r20, 0x10	; 16
     e78:	50 e0       	ldi	r21, 0x00	; 0
     e7a:	0e 94 bc 09 	call	0x1378	; 0x1378 <itoa>
     e7e:	80 e1       	ldi	r24, 0x10	; 16
     e80:	91 e2       	ldi	r25, 0x21	; 33
     e82:	6d e0       	ldi	r22, 0x0D	; 13
     e84:	0e 94 e0 02 	call	0x5c0	; 0x5c0 <USBUartSendArray>
     e88:	c7 01       	movw	r24, r14
     e8a:	64 e0       	ldi	r22, 0x04	; 4
     e8c:	0e 94 45 02 	call	0x48a	; 0x48a <DAC_2636WriteSingleChannel>
     e90:	e0 92 30 20 	sts	0x2030, r14
     e94:	f0 92 31 20 	sts	0x2031, r15
     e98:	80 e0       	ldi	r24, 0x00	; 0
     e9a:	2c c0       	rjmp	.+88     	; 0xef4 <TerminalCommandsWithArgument+0x298>
     e9c:	fa 01       	movw	r30, r20
     e9e:	e6 0f       	add	r30, r22
     ea0:	f1 1d       	adc	r31, r1
     ea2:	90 83       	st	Z, r25
     ea4:	ca 01       	movw	r24, r20
     ea6:	60 e0       	ldi	r22, 0x00	; 0
     ea8:	70 e0       	ldi	r23, 0x00	; 0
     eaa:	40 e1       	ldi	r20, 0x10	; 16
     eac:	50 e0       	ldi	r21, 0x00	; 0
     eae:	0e 94 9e 08 	call	0x113c	; 0x113c <strtoul>
     eb2:	7b 01       	movw	r14, r22
     eb4:	8c 01       	movw	r16, r24
     eb6:	80 e0       	ldi	r24, 0x00	; 0
     eb8:	e8 16       	cp	r14, r24
     eba:	80 e1       	ldi	r24, 0x10	; 16
     ebc:	f8 06       	cpc	r15, r24
     ebe:	80 e0       	ldi	r24, 0x00	; 0
     ec0:	08 07       	cpc	r16, r24
     ec2:	80 e0       	ldi	r24, 0x00	; 0
     ec4:	18 07       	cpc	r17, r24
     ec6:	a8 f4       	brcc	.+42     	; 0xef2 <TerminalCommandsWithArgument+0x296>
     ec8:	c7 01       	movw	r24, r14
     eca:	61 e1       	ldi	r22, 0x11	; 17
     ecc:	71 e2       	ldi	r23, 0x21	; 33
     ece:	40 e1       	ldi	r20, 0x10	; 16
     ed0:	50 e0       	ldi	r21, 0x00	; 0
     ed2:	0e 94 bc 09 	call	0x1378	; 0x1378 <itoa>
     ed6:	80 e1       	ldi	r24, 0x10	; 16
     ed8:	91 e2       	ldi	r25, 0x21	; 33
     eda:	6d e0       	ldi	r22, 0x0D	; 13
     edc:	0e 94 e0 02 	call	0x5c0	; 0x5c0 <USBUartSendArray>
     ee0:	c7 01       	movw	r24, r14
     ee2:	65 e0       	ldi	r22, 0x05	; 5
     ee4:	0e 94 45 02 	call	0x48a	; 0x48a <DAC_2636WriteSingleChannel>
     ee8:	e0 92 32 20 	sts	0x2032, r14
     eec:	f0 92 33 20 	sts	0x2033, r15
     ef0:	d3 cf       	rjmp	.-90     	; 0xe98 <TerminalCommandsWithArgument+0x23c>
     ef2:	81 e0       	ldi	r24, 0x01	; 1
     ef4:	1f 91       	pop	r17
     ef6:	0f 91       	pop	r16
     ef8:	ff 90       	pop	r15
     efa:	ef 90       	pop	r14
     efc:	08 95       	ret

00000efe <TerminalHandler>:
     efe:	1f 93       	push	r17
     f00:	18 2f       	mov	r17, r24
     f02:	8d 30       	cpi	r24, 0x0D	; 13
     f04:	21 f0       	breq	.+8      	; 0xf0e <TerminalHandler+0x10>
     f06:	8a 30       	cpi	r24, 0x0A	; 10
     f08:	11 f0       	breq	.+4      	; 0xf0e <TerminalHandler+0x10>
     f0a:	0e 94 45 03 	call	0x68a	; 0x68a <USBUartSendByte>
     f0e:	80 91 31 21 	lds	r24, 0x2131
     f12:	90 91 32 21 	lds	r25, 0x2132
     f16:	81 30       	cpi	r24, 0x01	; 1
     f18:	91 05       	cpc	r25, r1
     f1a:	b9 f0       	breq	.+46     	; 0xf4a <TerminalHandler+0x4c>
     f1c:	81 30       	cpi	r24, 0x01	; 1
     f1e:	91 05       	cpc	r25, r1
     f20:	38 f0       	brcs	.+14     	; 0xf30 <TerminalHandler+0x32>
     f22:	82 30       	cpi	r24, 0x02	; 2
     f24:	91 05       	cpc	r25, r1
     f26:	01 f1       	breq	.+64     	; 0xf68 <TerminalHandler+0x6a>
     f28:	03 97       	sbiw	r24, 0x03	; 3
     f2a:	09 f0       	breq	.+2      	; 0xf2e <TerminalHandler+0x30>
     f2c:	54 c0       	rjmp	.+168    	; 0xfd6 <TerminalHandler+0xd8>
     f2e:	33 c0       	rjmp	.+102    	; 0xf96 <TerminalHandler+0x98>
     f30:	10 92 24 21 	sts	0x2124, r1
     f34:	1d 30       	cpi	r17, 0x0D	; 13
     f36:	09 f4       	brne	.+2      	; 0xf3a <TerminalHandler+0x3c>
     f38:	52 c0       	rjmp	.+164    	; 0xfde <TerminalHandler+0xe0>
     f3a:	1a 30       	cpi	r17, 0x0A	; 10
     f3c:	09 f4       	brne	.+2      	; 0xf40 <TerminalHandler+0x42>
     f3e:	4f c0       	rjmp	.+158    	; 0xfde <TerminalHandler+0xe0>
     f40:	10 93 2f 21 	sts	0x212F, r17
     f44:	81 e0       	ldi	r24, 0x01	; 1
     f46:	90 e0       	ldi	r25, 0x00	; 0
     f48:	0a c0       	rjmp	.+20     	; 0xf5e <TerminalHandler+0x60>
     f4a:	1d 30       	cpi	r17, 0x0D	; 13
     f4c:	09 f4       	brne	.+2      	; 0xf50 <TerminalHandler+0x52>
     f4e:	43 c0       	rjmp	.+134    	; 0xfd6 <TerminalHandler+0xd8>
     f50:	1a 30       	cpi	r17, 0x0A	; 10
     f52:	09 f4       	brne	.+2      	; 0xf56 <TerminalHandler+0x58>
     f54:	40 c0       	rjmp	.+128    	; 0xfd6 <TerminalHandler+0xd8>
     f56:	10 93 30 21 	sts	0x2130, r17
     f5a:	82 e0       	ldi	r24, 0x02	; 2
     f5c:	90 e0       	ldi	r25, 0x00	; 0
     f5e:	80 93 31 21 	sts	0x2131, r24
     f62:	90 93 32 21 	sts	0x2132, r25
     f66:	40 c0       	rjmp	.+128    	; 0xfe8 <TerminalHandler+0xea>
     f68:	10 32       	cpi	r17, 0x20	; 32
     f6a:	91 f0       	breq	.+36     	; 0xf90 <TerminalHandler+0x92>
     f6c:	1d 30       	cpi	r17, 0x0D	; 13
     f6e:	11 f0       	breq	.+4      	; 0xf74 <TerminalHandler+0x76>
     f70:	1a 30       	cpi	r17, 0x0A	; 10
     f72:	21 f4       	brne	.+8      	; 0xf7c <TerminalHandler+0x7e>
     f74:	8f e2       	ldi	r24, 0x2F	; 47
     f76:	91 e2       	ldi	r25, 0x21	; 33
     f78:	0e 94 fa 04 	call	0x9f4	; 0x9f4 <TerminalCommandsNoArgument>
     f7c:	84 e2       	ldi	r24, 0x24	; 36
     f7e:	90 e2       	ldi	r25, 0x20	; 32
     f80:	64 e0       	ldi	r22, 0x04	; 4
     f82:	0e 94 e0 02 	call	0x5c0	; 0x5c0 <USBUartSendArray>
     f86:	10 92 31 21 	sts	0x2131, r1
     f8a:	10 92 32 21 	sts	0x2132, r1
     f8e:	2c c0       	rjmp	.+88     	; 0xfe8 <TerminalHandler+0xea>
     f90:	83 e0       	ldi	r24, 0x03	; 3
     f92:	90 e0       	ldi	r25, 0x00	; 0
     f94:	e4 cf       	rjmp	.-56     	; 0xf5e <TerminalHandler+0x60>
     f96:	1d 30       	cpi	r17, 0x0D	; 13
     f98:	11 f0       	breq	.+4      	; 0xf9e <TerminalHandler+0xa0>
     f9a:	1a 30       	cpi	r17, 0x0A	; 10
     f9c:	79 f4       	brne	.+30     	; 0xfbc <TerminalHandler+0xbe>
     f9e:	10 92 31 21 	sts	0x2131, r1
     fa2:	10 92 32 21 	sts	0x2132, r1
     fa6:	8f e2       	ldi	r24, 0x2F	; 47
     fa8:	91 e2       	ldi	r25, 0x21	; 33
     faa:	60 91 24 21 	lds	r22, 0x2124
     fae:	45 e2       	ldi	r20, 0x25	; 37
     fb0:	51 e2       	ldi	r21, 0x21	; 33
     fb2:	0e 94 2e 06 	call	0xc5c	; 0xc5c <TerminalCommandsWithArgument>
     fb6:	88 23       	and	r24, r24
     fb8:	b9 f0       	breq	.+46     	; 0xfe8 <TerminalHandler+0xea>
     fba:	11 c0       	rjmp	.+34     	; 0xfde <TerminalHandler+0xe0>
     fbc:	80 91 24 21 	lds	r24, 0x2124
     fc0:	8a 30       	cpi	r24, 0x0A	; 10
     fc2:	90 f4       	brcc	.+36     	; 0xfe8 <TerminalHandler+0xea>
     fc4:	e8 2f       	mov	r30, r24
     fc6:	f0 e0       	ldi	r31, 0x00	; 0
     fc8:	eb 5d       	subi	r30, 0xDB	; 219
     fca:	fe 4d       	sbci	r31, 0xDE	; 222
     fcc:	10 83       	st	Z, r17
     fce:	8f 5f       	subi	r24, 0xFF	; 255
     fd0:	80 93 24 21 	sts	0x2124, r24
     fd4:	09 c0       	rjmp	.+18     	; 0xfe8 <TerminalHandler+0xea>
     fd6:	10 92 31 21 	sts	0x2131, r1
     fda:	10 92 32 21 	sts	0x2132, r1
     fde:	84 e2       	ldi	r24, 0x24	; 36
     fe0:	90 e2       	ldi	r25, 0x20	; 32
     fe2:	64 e0       	ldi	r22, 0x04	; 4
     fe4:	0e 94 e0 02 	call	0x5c0	; 0x5c0 <USBUartSendArray>
     fe8:	1f 91       	pop	r17
     fea:	08 95       	ret

00000fec <main>:
     fec:	ff 92       	push	r15
     fee:	0f 93       	push	r16
     ff0:	1f 93       	push	r17
     ff2:	df 93       	push	r29
     ff4:	cf 93       	push	r28
     ff6:	cd b7       	in	r28, 0x3d	; 61
     ff8:	de b7       	in	r29, 0x3e	; 62
     ffa:	2c 97       	sbiw	r28, 0x0c	; 12
     ffc:	cd bf       	out	0x3d, r28	; 61
     ffe:	de bf       	out	0x3e, r29	; 62
    1000:	ce 01       	movw	r24, r28
    1002:	01 96       	adiw	r24, 0x01	; 1
    1004:	80 93 89 21 	sts	0x2189, r24
    1008:	90 93 8a 21 	sts	0x218A, r25
    100c:	0e 94 ad 03 	call	0x75a	; 0x75a <InitPorts>
    1010:	e0 e0       	ldi	r30, 0x00	; 0
    1012:	f6 e0       	ldi	r31, 0x06	; 6
    1014:	12 e0       	ldi	r17, 0x02	; 2
    1016:	15 83       	std	Z+5, r17	; 0x05
    1018:	81 e0       	ldi	r24, 0x01	; 1
    101a:	85 83       	std	Z+5, r24	; 0x05
    101c:	0e 94 da 03 	call	0x7b4	; 0x7b4 <SetClock>
    1020:	0e 94 32 03 	call	0x664	; 0x664 <USBUartInit>
    1024:	0e 94 22 03 	call	0x644	; 0x644 <USBUartDMASetup>
    1028:	88 ed       	ldi	r24, 0xD8	; 216
    102a:	84 bf       	out	0x34, r24	; 52
    102c:	80 91 80 00 	lds	r24, 0x0080
    1030:	8d 7f       	andi	r24, 0xFD	; 253
    1032:	80 93 80 00 	sts	0x0080, r24
    1036:	e0 e4       	ldi	r30, 0x40	; 64
    1038:	f6 e0       	ldi	r31, 0x06	; 6
    103a:	15 83       	std	Z+5, r17	; 0x05
    103c:	80 91 a2 00 	lds	r24, 0x00A2
    1040:	85 60       	ori	r24, 0x05	; 5
    1042:	e0 ea       	ldi	r30, 0xA0	; 160
    1044:	f0 e0       	ldi	r31, 0x00	; 0
    1046:	82 83       	std	Z+2, r24	; 0x02
    1048:	0e 94 6f 02 	call	0x4de	; 0x4de <DAC_2636_init>
    104c:	0e 94 7c 02 	call	0x4f8	; 0x4f8 <ADC_1408_init>
    1050:	78 94       	sei
    1052:	84 e6       	ldi	r24, 0x64	; 100
    1054:	90 e0       	ldi	r25, 0x00	; 0
    1056:	20 e2       	ldi	r18, 0x20	; 32
    1058:	33 e0       	ldi	r19, 0x03	; 3
    105a:	f9 01       	movw	r30, r18
    105c:	31 97       	sbiw	r30, 0x01	; 1
    105e:	f1 f7       	brne	.-4      	; 0x105c <main+0x70>
    1060:	01 97       	sbiw	r24, 0x01	; 1
    1062:	d9 f7       	brne	.-10     	; 0x105a <main+0x6e>
    1064:	0e 94 fe 03 	call	0x7fc	; 0x7fc <SetTimer>
    1068:	83 e8       	ldi	r24, 0x83	; 131
    106a:	80 93 00 01 	sts	0x0100, r24
    106e:	e0 e0       	ldi	r30, 0x00	; 0
    1070:	f6 e0       	ldi	r31, 0x06	; 6
    1072:	82 e0       	ldi	r24, 0x02	; 2
    1074:	86 83       	std	Z+6, r24	; 0x06
    1076:	81 e0       	ldi	r24, 0x01	; 1
    1078:	86 83       	std	Z+6, r24	; 0x06
    107a:	84 e2       	ldi	r24, 0x24	; 36
    107c:	90 e2       	ldi	r25, 0x20	; 32
    107e:	64 e0       	ldi	r22, 0x04	; 4
    1080:	0e 94 e0 02 	call	0x5c0	; 0x5c0 <USBUartSendArray>
    1084:	00 e0       	ldi	r16, 0x00	; 0
    1086:	16 e0       	ldi	r17, 0x06	; 6
    1088:	ff 24       	eor	r15, r15
    108a:	f3 94       	inc	r15
    108c:	0e 94 c3 02 	call	0x586	; 0x586 <USBUartRXQuelength>
    1090:	88 23       	and	r24, r24
    1092:	21 f0       	breq	.+8      	; 0x109c <main+0xb0>
    1094:	0e 94 c6 02 	call	0x58c	; 0x58c <USBUartReadByteFromBuffer>
    1098:	0e 94 7f 07 	call	0xefe	; 0xefe <TerminalHandler>
    109c:	0e 94 8e 01 	call	0x31c	; 0x31c <SPITransferReady>
    10a0:	88 23       	and	r24, r24
    10a2:	51 f0       	breq	.+20     	; 0x10b8 <main+0xcc>
    10a4:	0e 94 94 01 	call	0x328	; 0x328 <SPITarget>
    10a8:	89 2b       	or	r24, r25
    10aa:	31 f4       	brne	.+12     	; 0x10b8 <main+0xcc>
    10ac:	0e 94 8b 01 	call	0x316	; 0x316 <SPIbufferpointer>
    10b0:	64 ed       	ldi	r22, 0xD4	; 212
    10b2:	72 e2       	ldi	r23, 0x22	; 34
    10b4:	0e 94 78 03 	call	0x6f0	; 0x6f0 <ConvertADCResults>
    10b8:	0e 94 9a 01 	call	0x334	; 0x334 <SPIClearBuffer>
    10bc:	80 91 6a 23 	lds	r24, 0x236A
    10c0:	88 23       	and	r24, r24
    10c2:	21 f3       	breq	.-56     	; 0x108c <main+0xa0>
    10c4:	f8 01       	movw	r30, r16
    10c6:	f5 82       	std	Z+5, r15	; 0x05
    10c8:	e1 cf       	rjmp	.-62     	; 0x108c <main+0xa0>

000010ca <__vector_16>:
    10ca:	1f 92       	push	r1
    10cc:	0f 92       	push	r0
    10ce:	0f b6       	in	r0, 0x3f	; 63
    10d0:	0f 92       	push	r0
    10d2:	08 b6       	in	r0, 0x38	; 56
    10d4:	0f 92       	push	r0
    10d6:	09 b6       	in	r0, 0x39	; 57
    10d8:	0f 92       	push	r0
    10da:	0b b6       	in	r0, 0x3b	; 59
    10dc:	0f 92       	push	r0
    10de:	11 24       	eor	r1, r1
    10e0:	18 be       	out	0x38, r1	; 56
    10e2:	19 be       	out	0x39, r1	; 57
    10e4:	1b be       	out	0x3b, r1	; 59
    10e6:	2f 93       	push	r18
    10e8:	3f 93       	push	r19
    10ea:	4f 93       	push	r20
    10ec:	5f 93       	push	r21
    10ee:	6f 93       	push	r22
    10f0:	7f 93       	push	r23
    10f2:	8f 93       	push	r24
    10f4:	9f 93       	push	r25
    10f6:	af 93       	push	r26
    10f8:	bf 93       	push	r27
    10fa:	ef 93       	push	r30
    10fc:	ff 93       	push	r31
    10fe:	80 91 89 21 	lds	r24, 0x2189
    1102:	90 91 8a 21 	lds	r25, 0x218A
    1106:	6c e0       	ldi	r22, 0x0C	; 12
    1108:	40 e0       	ldi	r20, 0x00	; 0
    110a:	0e 94 ca 01 	call	0x394	; 0x394 <SPITransceiveArray>
    110e:	ff 91       	pop	r31
    1110:	ef 91       	pop	r30
    1112:	bf 91       	pop	r27
    1114:	af 91       	pop	r26
    1116:	9f 91       	pop	r25
    1118:	8f 91       	pop	r24
    111a:	7f 91       	pop	r23
    111c:	6f 91       	pop	r22
    111e:	5f 91       	pop	r21
    1120:	4f 91       	pop	r20
    1122:	3f 91       	pop	r19
    1124:	2f 91       	pop	r18
    1126:	0f 90       	pop	r0
    1128:	0b be       	out	0x3b, r0	; 59
    112a:	0f 90       	pop	r0
    112c:	09 be       	out	0x39, r0	; 57
    112e:	0f 90       	pop	r0
    1130:	08 be       	out	0x38, r0	; 56
    1132:	0f 90       	pop	r0
    1134:	0f be       	out	0x3f, r0	; 63
    1136:	0f 90       	pop	r0
    1138:	1f 90       	pop	r1
    113a:	18 95       	reti

0000113c <strtoul>:
    113c:	3f 92       	push	r3
    113e:	4f 92       	push	r4
    1140:	5f 92       	push	r5
    1142:	6f 92       	push	r6
    1144:	7f 92       	push	r7
    1146:	8f 92       	push	r8
    1148:	9f 92       	push	r9
    114a:	af 92       	push	r10
    114c:	bf 92       	push	r11
    114e:	cf 92       	push	r12
    1150:	df 92       	push	r13
    1152:	ef 92       	push	r14
    1154:	ff 92       	push	r15
    1156:	0f 93       	push	r16
    1158:	1f 93       	push	r17
    115a:	cf 93       	push	r28
    115c:	df 93       	push	r29
    115e:	ec 01       	movw	r28, r24
    1160:	2b 01       	movw	r4, r22
    1162:	6a 01       	movw	r12, r20
    1164:	61 15       	cp	r22, r1
    1166:	71 05       	cpc	r23, r1
    1168:	19 f0       	breq	.+6      	; 0x1170 <strtoul+0x34>
    116a:	fb 01       	movw	r30, r22
    116c:	80 83       	st	Z, r24
    116e:	91 83       	std	Z+1, r25	; 0x01
    1170:	c1 14       	cp	r12, r1
    1172:	d1 04       	cpc	r13, r1
    1174:	49 f0       	breq	.+18     	; 0x1188 <strtoul+0x4c>
    1176:	c6 01       	movw	r24, r12
    1178:	02 97       	sbiw	r24, 0x02	; 2
    117a:	83 97       	sbiw	r24, 0x23	; 35
    117c:	28 f0       	brcs	.+10     	; 0x1188 <strtoul+0x4c>
    117e:	20 e0       	ldi	r18, 0x00	; 0
    1180:	30 e0       	ldi	r19, 0x00	; 0
    1182:	40 e0       	ldi	r20, 0x00	; 0
    1184:	50 e0       	ldi	r21, 0x00	; 0
    1186:	dc c0       	rjmp	.+440    	; 0x1340 <strtoul+0x204>
    1188:	a9 90       	ld	r10, Y+
    118a:	8a 2d       	mov	r24, r10
    118c:	90 e0       	ldi	r25, 0x00	; 0
    118e:	0e 94 b4 09 	call	0x1368	; 0x1368 <isspace>
    1192:	89 2b       	or	r24, r25
    1194:	c9 f7       	brne	.-14     	; 0x1188 <strtoul+0x4c>
    1196:	fd e2       	ldi	r31, 0x2D	; 45
    1198:	af 16       	cp	r10, r31
    119a:	21 f4       	brne	.+8      	; 0x11a4 <strtoul+0x68>
    119c:	a9 90       	ld	r10, Y+
    119e:	33 24       	eor	r3, r3
    11a0:	33 94       	inc	r3
    11a2:	05 c0       	rjmp	.+10     	; 0x11ae <strtoul+0x72>
    11a4:	8b e2       	ldi	r24, 0x2B	; 43
    11a6:	a8 16       	cp	r10, r24
    11a8:	09 f4       	brne	.+2      	; 0x11ac <strtoul+0x70>
    11aa:	a9 90       	ld	r10, Y+
    11ac:	33 24       	eor	r3, r3
    11ae:	c1 14       	cp	r12, r1
    11b0:	d1 04       	cpc	r13, r1
    11b2:	21 f0       	breq	.+8      	; 0x11bc <strtoul+0x80>
    11b4:	e0 e1       	ldi	r30, 0x10	; 16
    11b6:	ce 16       	cp	r12, r30
    11b8:	d1 04       	cpc	r13, r1
    11ba:	11 f5       	brne	.+68     	; 0x1200 <strtoul+0xc4>
    11bc:	f0 e3       	ldi	r31, 0x30	; 48
    11be:	af 16       	cp	r10, r31
    11c0:	69 f4       	brne	.+26     	; 0x11dc <strtoul+0xa0>
    11c2:	88 81       	ld	r24, Y
    11c4:	88 37       	cpi	r24, 0x78	; 120
    11c6:	11 f0       	breq	.+4      	; 0x11cc <strtoul+0x90>
    11c8:	88 35       	cpi	r24, 0x58	; 88
    11ca:	41 f4       	brne	.+16     	; 0x11dc <strtoul+0xa0>
    11cc:	a9 80       	ldd	r10, Y+1	; 0x01
    11ce:	22 96       	adiw	r28, 0x02	; 2
    11d0:	82 e0       	ldi	r24, 0x02	; 2
    11d2:	38 2a       	or	r3, r24
    11d4:	20 e1       	ldi	r18, 0x10	; 16
    11d6:	c2 2e       	mov	r12, r18
    11d8:	d1 2c       	mov	r13, r1
    11da:	12 c0       	rjmp	.+36     	; 0x1200 <strtoul+0xc4>
    11dc:	c1 14       	cp	r12, r1
    11de:	d1 04       	cpc	r13, r1
    11e0:	79 f4       	brne	.+30     	; 0x1200 <strtoul+0xc4>
    11e2:	e0 e3       	ldi	r30, 0x30	; 48
    11e4:	ae 16       	cp	r10, r30
    11e6:	59 f1       	breq	.+86     	; 0x123e <strtoul+0x102>
    11e8:	99 e9       	ldi	r25, 0x99	; 153
    11ea:	e9 2e       	mov	r14, r25
    11ec:	99 e9       	ldi	r25, 0x99	; 153
    11ee:	f9 2e       	mov	r15, r25
    11f0:	99 e9       	ldi	r25, 0x99	; 153
    11f2:	09 2f       	mov	r16, r25
    11f4:	99 e1       	ldi	r25, 0x19	; 25
    11f6:	19 2f       	mov	r17, r25
    11f8:	8a e0       	ldi	r24, 0x0A	; 10
    11fa:	c8 2e       	mov	r12, r24
    11fc:	d1 2c       	mov	r13, r1
    11fe:	3a c0       	rjmp	.+116    	; 0x1274 <strtoul+0x138>
    1200:	fa e0       	ldi	r31, 0x0A	; 10
    1202:	cf 16       	cp	r12, r31
    1204:	d1 04       	cpc	r13, r1
    1206:	91 f0       	breq	.+36     	; 0x122c <strtoul+0xf0>
    1208:	80 e1       	ldi	r24, 0x10	; 16
    120a:	c8 16       	cp	r12, r24
    120c:	d1 04       	cpc	r13, r1
    120e:	29 f0       	breq	.+10     	; 0x121a <strtoul+0xde>
    1210:	e8 e0       	ldi	r30, 0x08	; 8
    1212:	ce 16       	cp	r12, r30
    1214:	d1 04       	cpc	r13, r1
    1216:	f9 f4       	brne	.+62     	; 0x1256 <strtoul+0x11a>
    1218:	15 c0       	rjmp	.+42     	; 0x1244 <strtoul+0x108>
    121a:	bf ef       	ldi	r27, 0xFF	; 255
    121c:	eb 2e       	mov	r14, r27
    121e:	bf ef       	ldi	r27, 0xFF	; 255
    1220:	fb 2e       	mov	r15, r27
    1222:	bf ef       	ldi	r27, 0xFF	; 255
    1224:	0b 2f       	mov	r16, r27
    1226:	bf e0       	ldi	r27, 0x0F	; 15
    1228:	1b 2f       	mov	r17, r27
    122a:	24 c0       	rjmp	.+72     	; 0x1274 <strtoul+0x138>
    122c:	a9 e9       	ldi	r26, 0x99	; 153
    122e:	ea 2e       	mov	r14, r26
    1230:	a9 e9       	ldi	r26, 0x99	; 153
    1232:	fa 2e       	mov	r15, r26
    1234:	a9 e9       	ldi	r26, 0x99	; 153
    1236:	0a 2f       	mov	r16, r26
    1238:	a9 e1       	ldi	r26, 0x19	; 25
    123a:	1a 2f       	mov	r17, r26
    123c:	1b c0       	rjmp	.+54     	; 0x1274 <strtoul+0x138>
    123e:	f8 e0       	ldi	r31, 0x08	; 8
    1240:	cf 2e       	mov	r12, r31
    1242:	d1 2c       	mov	r13, r1
    1244:	ef ef       	ldi	r30, 0xFF	; 255
    1246:	ee 2e       	mov	r14, r30
    1248:	ef ef       	ldi	r30, 0xFF	; 255
    124a:	fe 2e       	mov	r15, r30
    124c:	ef ef       	ldi	r30, 0xFF	; 255
    124e:	0e 2f       	mov	r16, r30
    1250:	ef e1       	ldi	r30, 0x1F	; 31
    1252:	1e 2f       	mov	r17, r30
    1254:	0f c0       	rjmp	.+30     	; 0x1274 <strtoul+0x138>
    1256:	96 01       	movw	r18, r12
    1258:	44 27       	eor	r20, r20
    125a:	37 fd       	sbrc	r19, 7
    125c:	40 95       	com	r20
    125e:	54 2f       	mov	r21, r20
    1260:	6f ef       	ldi	r22, 0xFF	; 255
    1262:	7f ef       	ldi	r23, 0xFF	; 255
    1264:	8f ef       	ldi	r24, 0xFF	; 255
    1266:	9f ef       	ldi	r25, 0xFF	; 255
    1268:	0e 94 23 0a 	call	0x1446	; 0x1446 <__udivmodsi4>
    126c:	c9 01       	movw	r24, r18
    126e:	da 01       	movw	r26, r20
    1270:	7c 01       	movw	r14, r24
    1272:	8d 01       	movw	r16, r26
    1274:	20 e0       	ldi	r18, 0x00	; 0
    1276:	30 e0       	ldi	r19, 0x00	; 0
    1278:	40 e0       	ldi	r20, 0x00	; 0
    127a:	50 e0       	ldi	r21, 0x00	; 0
    127c:	60 e0       	ldi	r22, 0x00	; 0
    127e:	36 01       	movw	r6, r12
    1280:	88 24       	eor	r8, r8
    1282:	77 fc       	sbrc	r7, 7
    1284:	80 94       	com	r8
    1286:	98 2c       	mov	r9, r8
    1288:	70 ed       	ldi	r23, 0xD0	; 208
    128a:	b7 2e       	mov	r11, r23
    128c:	ba 0c       	add	r11, r10
    128e:	f9 e0       	ldi	r31, 0x09	; 9
    1290:	fb 15       	cp	r31, r11
    1292:	70 f4       	brcc	.+28     	; 0x12b0 <strtoul+0x174>
    1294:	8a 2d       	mov	r24, r10
    1296:	81 54       	subi	r24, 0x41	; 65
    1298:	8a 31       	cpi	r24, 0x1A	; 26
    129a:	18 f4       	brcc	.+6      	; 0x12a2 <strtoul+0x166>
    129c:	99 ec       	ldi	r25, 0xC9	; 201
    129e:	b9 2e       	mov	r11, r25
    12a0:	06 c0       	rjmp	.+12     	; 0x12ae <strtoul+0x172>
    12a2:	8a 2d       	mov	r24, r10
    12a4:	81 56       	subi	r24, 0x61	; 97
    12a6:	8a 31       	cpi	r24, 0x1A	; 26
    12a8:	48 f5       	brcc	.+82     	; 0x12fc <strtoul+0x1c0>
    12aa:	89 ea       	ldi	r24, 0xA9	; 169
    12ac:	b8 2e       	mov	r11, r24
    12ae:	ba 0c       	add	r11, r10
    12b0:	8b 2d       	mov	r24, r11
    12b2:	90 e0       	ldi	r25, 0x00	; 0
    12b4:	8c 15       	cp	r24, r12
    12b6:	9d 05       	cpc	r25, r13
    12b8:	0c f5       	brge	.+66     	; 0x12fc <strtoul+0x1c0>
    12ba:	6f 3f       	cpi	r22, 0xFF	; 255
    12bc:	e9 f0       	breq	.+58     	; 0x12f8 <strtoul+0x1bc>
    12be:	e2 16       	cp	r14, r18
    12c0:	f3 06       	cpc	r15, r19
    12c2:	04 07       	cpc	r16, r20
    12c4:	15 07       	cpc	r17, r21
    12c6:	b8 f0       	brcs	.+46     	; 0x12f6 <strtoul+0x1ba>
    12c8:	ca 01       	movw	r24, r20
    12ca:	b9 01       	movw	r22, r18
    12cc:	a4 01       	movw	r20, r8
    12ce:	93 01       	movw	r18, r6
    12d0:	0e 94 f0 09 	call	0x13e0	; 0x13e0 <__mulsi3>
    12d4:	9b 01       	movw	r18, r22
    12d6:	ac 01       	movw	r20, r24
    12d8:	8b 2d       	mov	r24, r11
    12da:	90 e0       	ldi	r25, 0x00	; 0
    12dc:	a0 e0       	ldi	r26, 0x00	; 0
    12de:	b0 e0       	ldi	r27, 0x00	; 0
    12e0:	28 0f       	add	r18, r24
    12e2:	39 1f       	adc	r19, r25
    12e4:	4a 1f       	adc	r20, r26
    12e6:	5b 1f       	adc	r21, r27
    12e8:	28 17       	cp	r18, r24
    12ea:	39 07       	cpc	r19, r25
    12ec:	4a 07       	cpc	r20, r26
    12ee:	5b 07       	cpc	r21, r27
    12f0:	10 f0       	brcs	.+4      	; 0x12f6 <strtoul+0x1ba>
    12f2:	61 e0       	ldi	r22, 0x01	; 1
    12f4:	01 c0       	rjmp	.+2      	; 0x12f8 <strtoul+0x1bc>
    12f6:	6f ef       	ldi	r22, 0xFF	; 255
    12f8:	a9 90       	ld	r10, Y+
    12fa:	c6 cf       	rjmp	.-116    	; 0x1288 <strtoul+0x14c>
    12fc:	41 14       	cp	r4, r1
    12fe:	51 04       	cpc	r5, r1
    1300:	51 f0       	breq	.+20     	; 0x1316 <strtoul+0x1da>
    1302:	66 23       	and	r22, r22
    1304:	11 f0       	breq	.+4      	; 0x130a <strtoul+0x1ce>
    1306:	21 97       	sbiw	r28, 0x01	; 1
    1308:	03 c0       	rjmp	.+6      	; 0x1310 <strtoul+0x1d4>
    130a:	31 fe       	sbrs	r3, 1
    130c:	04 c0       	rjmp	.+8      	; 0x1316 <strtoul+0x1da>
    130e:	22 97       	sbiw	r28, 0x02	; 2
    1310:	f2 01       	movw	r30, r4
    1312:	c0 83       	st	Z, r28
    1314:	d1 83       	std	Z+1, r29	; 0x01
    1316:	30 fe       	sbrs	r3, 0
    1318:	07 c0       	rjmp	.+14     	; 0x1328 <strtoul+0x1ec>
    131a:	50 95       	com	r21
    131c:	40 95       	com	r20
    131e:	30 95       	com	r19
    1320:	21 95       	neg	r18
    1322:	3f 4f       	sbci	r19, 0xFF	; 255
    1324:	4f 4f       	sbci	r20, 0xFF	; 255
    1326:	5f 4f       	sbci	r21, 0xFF	; 255
    1328:	67 ff       	sbrs	r22, 7
    132a:	0a c0       	rjmp	.+20     	; 0x1340 <strtoul+0x204>
    132c:	82 e2       	ldi	r24, 0x22	; 34
    132e:	90 e0       	ldi	r25, 0x00	; 0
    1330:	80 93 6d 23 	sts	0x236D, r24
    1334:	90 93 6e 23 	sts	0x236E, r25
    1338:	2f ef       	ldi	r18, 0xFF	; 255
    133a:	3f ef       	ldi	r19, 0xFF	; 255
    133c:	4f ef       	ldi	r20, 0xFF	; 255
    133e:	5f ef       	ldi	r21, 0xFF	; 255
    1340:	b9 01       	movw	r22, r18
    1342:	ca 01       	movw	r24, r20
    1344:	df 91       	pop	r29
    1346:	cf 91       	pop	r28
    1348:	1f 91       	pop	r17
    134a:	0f 91       	pop	r16
    134c:	ff 90       	pop	r15
    134e:	ef 90       	pop	r14
    1350:	df 90       	pop	r13
    1352:	cf 90       	pop	r12
    1354:	bf 90       	pop	r11
    1356:	af 90       	pop	r10
    1358:	9f 90       	pop	r9
    135a:	8f 90       	pop	r8
    135c:	7f 90       	pop	r7
    135e:	6f 90       	pop	r6
    1360:	5f 90       	pop	r5
    1362:	4f 90       	pop	r4
    1364:	3f 90       	pop	r3
    1366:	08 95       	ret

00001368 <isspace>:
    1368:	91 11       	cpse	r25, r1
    136a:	27 c0       	rjmp	.+78     	; 0x13ba <__ctype_isfalse>
    136c:	80 32       	cpi	r24, 0x20	; 32
    136e:	19 f0       	breq	.+6      	; 0x1376 <isspace+0xe>
    1370:	89 50       	subi	r24, 0x09	; 9
    1372:	85 50       	subi	r24, 0x05	; 5
    1374:	d0 f7       	brcc	.-12     	; 0x136a <isspace+0x2>
    1376:	08 95       	ret

00001378 <itoa>:
    1378:	fb 01       	movw	r30, r22
    137a:	9f 01       	movw	r18, r30
    137c:	e8 94       	clt
    137e:	42 30       	cpi	r20, 0x02	; 2
    1380:	c4 f0       	brlt	.+48     	; 0x13b2 <itoa+0x3a>
    1382:	45 32       	cpi	r20, 0x25	; 37
    1384:	b4 f4       	brge	.+44     	; 0x13b2 <itoa+0x3a>
    1386:	4a 30       	cpi	r20, 0x0A	; 10
    1388:	29 f4       	brne	.+10     	; 0x1394 <itoa+0x1c>
    138a:	97 fb       	bst	r25, 7
    138c:	1e f4       	brtc	.+6      	; 0x1394 <itoa+0x1c>
    138e:	90 95       	com	r25
    1390:	81 95       	neg	r24
    1392:	9f 4f       	sbci	r25, 0xFF	; 255
    1394:	64 2f       	mov	r22, r20
    1396:	77 27       	eor	r23, r23
    1398:	0e 94 0f 0a 	call	0x141e	; 0x141e <__udivmodhi4>
    139c:	80 5d       	subi	r24, 0xD0	; 208
    139e:	8a 33       	cpi	r24, 0x3A	; 58
    13a0:	0c f0       	brlt	.+2      	; 0x13a4 <itoa+0x2c>
    13a2:	89 5d       	subi	r24, 0xD9	; 217
    13a4:	81 93       	st	Z+, r24
    13a6:	cb 01       	movw	r24, r22
    13a8:	00 97       	sbiw	r24, 0x00	; 0
    13aa:	a1 f7       	brne	.-24     	; 0x1394 <itoa+0x1c>
    13ac:	16 f4       	brtc	.+4      	; 0x13b2 <itoa+0x3a>
    13ae:	5d e2       	ldi	r21, 0x2D	; 45
    13b0:	51 93       	st	Z+, r21
    13b2:	10 82       	st	Z, r1
    13b4:	c9 01       	movw	r24, r18
    13b6:	0c 94 e0 09 	jmp	0x13c0	; 0x13c0 <strrev>

000013ba <__ctype_isfalse>:
    13ba:	99 27       	eor	r25, r25
    13bc:	88 27       	eor	r24, r24

000013be <__ctype_istrue>:
    13be:	08 95       	ret

000013c0 <strrev>:
    13c0:	dc 01       	movw	r26, r24
    13c2:	fc 01       	movw	r30, r24
    13c4:	67 2f       	mov	r22, r23
    13c6:	71 91       	ld	r23, Z+
    13c8:	77 23       	and	r23, r23
    13ca:	e1 f7       	brne	.-8      	; 0x13c4 <strrev+0x4>
    13cc:	32 97       	sbiw	r30, 0x02	; 2
    13ce:	04 c0       	rjmp	.+8      	; 0x13d8 <strrev+0x18>
    13d0:	7c 91       	ld	r23, X
    13d2:	6d 93       	st	X+, r22
    13d4:	70 83       	st	Z, r23
    13d6:	62 91       	ld	r22, -Z
    13d8:	ae 17       	cp	r26, r30
    13da:	bf 07       	cpc	r27, r31
    13dc:	c8 f3       	brcs	.-14     	; 0x13d0 <strrev+0x10>
    13de:	08 95       	ret

000013e0 <__mulsi3>:
    13e0:	62 9f       	mul	r22, r18
    13e2:	d0 01       	movw	r26, r0
    13e4:	73 9f       	mul	r23, r19
    13e6:	f0 01       	movw	r30, r0
    13e8:	82 9f       	mul	r24, r18
    13ea:	e0 0d       	add	r30, r0
    13ec:	f1 1d       	adc	r31, r1
    13ee:	64 9f       	mul	r22, r20
    13f0:	e0 0d       	add	r30, r0
    13f2:	f1 1d       	adc	r31, r1
    13f4:	92 9f       	mul	r25, r18
    13f6:	f0 0d       	add	r31, r0
    13f8:	83 9f       	mul	r24, r19
    13fa:	f0 0d       	add	r31, r0
    13fc:	74 9f       	mul	r23, r20
    13fe:	f0 0d       	add	r31, r0
    1400:	65 9f       	mul	r22, r21
    1402:	f0 0d       	add	r31, r0
    1404:	99 27       	eor	r25, r25
    1406:	72 9f       	mul	r23, r18
    1408:	b0 0d       	add	r27, r0
    140a:	e1 1d       	adc	r30, r1
    140c:	f9 1f       	adc	r31, r25
    140e:	63 9f       	mul	r22, r19
    1410:	b0 0d       	add	r27, r0
    1412:	e1 1d       	adc	r30, r1
    1414:	f9 1f       	adc	r31, r25
    1416:	bd 01       	movw	r22, r26
    1418:	cf 01       	movw	r24, r30
    141a:	11 24       	eor	r1, r1
    141c:	08 95       	ret

0000141e <__udivmodhi4>:
    141e:	aa 1b       	sub	r26, r26
    1420:	bb 1b       	sub	r27, r27
    1422:	51 e1       	ldi	r21, 0x11	; 17
    1424:	07 c0       	rjmp	.+14     	; 0x1434 <__udivmodhi4_ep>

00001426 <__udivmodhi4_loop>:
    1426:	aa 1f       	adc	r26, r26
    1428:	bb 1f       	adc	r27, r27
    142a:	a6 17       	cp	r26, r22
    142c:	b7 07       	cpc	r27, r23
    142e:	10 f0       	brcs	.+4      	; 0x1434 <__udivmodhi4_ep>
    1430:	a6 1b       	sub	r26, r22
    1432:	b7 0b       	sbc	r27, r23

00001434 <__udivmodhi4_ep>:
    1434:	88 1f       	adc	r24, r24
    1436:	99 1f       	adc	r25, r25
    1438:	5a 95       	dec	r21
    143a:	a9 f7       	brne	.-22     	; 0x1426 <__udivmodhi4_loop>
    143c:	80 95       	com	r24
    143e:	90 95       	com	r25
    1440:	bc 01       	movw	r22, r24
    1442:	cd 01       	movw	r24, r26
    1444:	08 95       	ret

00001446 <__udivmodsi4>:
    1446:	a1 e2       	ldi	r26, 0x21	; 33
    1448:	1a 2e       	mov	r1, r26
    144a:	aa 1b       	sub	r26, r26
    144c:	bb 1b       	sub	r27, r27
    144e:	fd 01       	movw	r30, r26
    1450:	0d c0       	rjmp	.+26     	; 0x146c <__udivmodsi4_ep>

00001452 <__udivmodsi4_loop>:
    1452:	aa 1f       	adc	r26, r26
    1454:	bb 1f       	adc	r27, r27
    1456:	ee 1f       	adc	r30, r30
    1458:	ff 1f       	adc	r31, r31
    145a:	a2 17       	cp	r26, r18
    145c:	b3 07       	cpc	r27, r19
    145e:	e4 07       	cpc	r30, r20
    1460:	f5 07       	cpc	r31, r21
    1462:	20 f0       	brcs	.+8      	; 0x146c <__udivmodsi4_ep>
    1464:	a2 1b       	sub	r26, r18
    1466:	b3 0b       	sbc	r27, r19
    1468:	e4 0b       	sbc	r30, r20
    146a:	f5 0b       	sbc	r31, r21

0000146c <__udivmodsi4_ep>:
    146c:	66 1f       	adc	r22, r22
    146e:	77 1f       	adc	r23, r23
    1470:	88 1f       	adc	r24, r24
    1472:	99 1f       	adc	r25, r25
    1474:	1a 94       	dec	r1
    1476:	69 f7       	brne	.-38     	; 0x1452 <__udivmodsi4_loop>
    1478:	60 95       	com	r22
    147a:	70 95       	com	r23
    147c:	80 95       	com	r24
    147e:	90 95       	com	r25
    1480:	9b 01       	movw	r18, r22
    1482:	ac 01       	movw	r20, r24
    1484:	bd 01       	movw	r22, r26
    1486:	cf 01       	movw	r24, r30
    1488:	08 95       	ret

0000148a <_exit>:
    148a:	f8 94       	cli

0000148c <__stop_program>:
    148c:	ff cf       	rjmp	.-2      	; 0x148c <__stop_program>
